:106679000000090200000301FA0400FA0500030AF8
:106689000A5A0B001E0C00FA0D00030E00040F013C
:1066990064100096120132130AFA14010217010A52
:1066A9001801FA1905321A010A1B01FA1C05321FD1
:1066B900FFFF20FFFF23011E2400642A00FA2B009C
:1066C900FA2C50782D003D2E004630006432507867
:1066D9003300003432FA3501643601643701503829
:1066E9000A643C00643E003C3F000140FFFF411446
:1066F90050420A5A430AC84405324500B44600FAD2
:106709004C00FA500404510596520A32530B465470
:106719000A96570546590A465A32FA5B010A5C0A33
:10672900325E000A5F00FE64021067FFFF6A0A3CDE
:106739006B00006C329673000174000178013279A4
:1067490001327E006481006484FFFF8A00019D0A92
:10675900969E00019FFFFFA00124A2000AA3FFFF4C
:10676900A4FFFFA5FFFFA6FFFFA7FFFFA8FFFFA943
:10677900FFFF0101481500022F003C47014848026C
:10678900035601044EFFFF58000261FFFF66000235
:106799008500AF8600018700FA89010A990008A1DE
:1067A90000FAFAFAFA0101241500022F1E3C4701EA
:1067B900484802035601034EFFFF58000261FFFFDC
:1067C9006600028500AF8600018700FA89010A99EF
:1067D9000000A10000FAFAFA0101241500002F1E99
:1067E9003C4701244802025601014EFFFF580000B0
:1067F90061FFFF66000085FFFF86FFFF87FFFF89B6
:106809000102990000A10000FAFAFA0065006F0080
:10681900790083008D009700A100AC00B600C0008C
:10682900CA00D400DE00E800F200580060006800E9
:10683900700078008000880090009800A000A800EF
:10684900B000B800C100C800D000D800DF00E600E1
:10685900EE00F600410047004D00530059005F006B
:1068690065006C00710077007D00830089008F004E
:1068790095009B00A200A700AC00B200B900C000BF
:0F688900C500CA00D200D500DD00E100E700EF36
:10331000900885E0900111F0900886E0900080F020
:10332000900887E09000A0F0900888E09000C9F035
:10333000900889E0900075F090088AE09000BBF05A
:1033400090088BE09000D9F090088CE09000ADF0F0
:1033500090088DE09000CBF090088EE09000FBF09C
:1033600090088FE090015FF0900890E0900160F08D
:10337000900891E0900161F090015FE0700C900185
:1033800060E07006900161E060028004C22080026B
:10339000D220743390014AF0743690014BF0742DB2
:1033A00090014CF0743290014DF0742090014EF079
:1033B000743490014FF07443900150F0747990018F
:1033C00051F0746C900152F07420900153F074200D
:1033D000900154F07420900155F07420900156F043
:1033E0007420900157F07420900158F02290087DCD
:1033F000E0FEA3E0FF7402D39F74019E400C906630
:1034000079120048E493F599804C90004BE0D394F6
:1034100005401490087DE0FEA3E0FF90667912005D
:1034200048E493F599802F90004BE0D39404401426
:1034300090087DE0FEA3E0FF9066AC120048E493A4
:10344000F599801290087DE0FEA3E0FF9066DF1200
:103450000048E493F59990087D1269B890087DE0E2
:10346000FEA3E0FFEFB43507EEB40103754D002273
:1034700085F97385FA747E017F00E5741269AAE507
:10348000732FFF50010E8E5A8F5B900015E0FCA346
:10349000E0FDEF2DFDEE3CFC8C5C8D5D2275A710F0
:1034A00085F97385FA747E017F00E5741269AAE5D7
:1034B000732FFF50010E8E5A8F5B9000D9E0B4023B
:1034C00010AC2CAD2DEF2DFDEE3CFC8C5C8D5D80A9
:1034D00016AE5AAF5B900015E0FCA3E0FDEF2DFDAA
:1034E000EE3CFC8C5C8D5D22AE5AAF5B740A8E04A0
:1034F0008F05FF12699A8C5C8D5DAE5AAF5B740AC2
:103500008E048F05FF1269C58C5A8D5BC200E55B86
:10351000455A6013740AC3955BFFE4955AFE8E5AB0
:103520008F5B785C1269FDE573A85CB80015D395D4
:103530005D4010E573C3955DFFE4955CFE8E5C8F86
:103540005D8012E5732424C3955DFFE4955CFE8ED7
:103550005C8F5DD200AE5CAF5D74236F4E6006740D
:10356000246F4E701AAE5CAF5D74236F4E7005759C
:1035700073018003757302755D22755C00800375AD
:10358000730022900087E0B40104C2078002D207D2
:10359000900088E0B40104C2088002D2089000C5FF
:1035A000E075F0E1A4FFAEF0740A8E048F05FF12FF
:1035B000699A900875ECF0A3EDF074078C068D07FE
:1035C0001269AA74038E048F05FF12699A90001184
:1035D000ECF0A3EDF07E017F00900083E01269AA79
:1035E0009000C6E08E048F05FF12699A740AFF12DC
:1035F000699A8D609000CFE075F0E1A4FFAEF074A1
:103600000A8E048F05FF12699A900879ECF0A3EDF9
:10361000F09000D1E060139000D1E0F5F0741684D2
:10362000FF7E00EF9008A1F0800674649008A1F07E
:103630009000C7E0900062F0900113E090006DF000
:10364000900115E0FE9000C3E08E0088F0A4FFAE6C
:10365000F0EF9008A9F0900111E0900885F090003B
:10366000A0E0900887F0900075E0900889F0900045
:10367000FBE090088EF090015FE090088FF09001E1
:1036800060E0900890F0900161E0900891F0A22035
:10369000B3401690015FE0700C900160E0700690FE
:1036A0000161E060028002C22090015FE0B4300F4F
:1036B000900160E0B44708900161E0643B600280E3
:1036C00004D2218002C22174E3900061F09000B026
:1036D000E0B40B0874E3900061F0805A9000B0E011
:1036E000B419129000C6E09067FF12008CE493902A
:1036F0000061F080419000B0E0B41E129000C6E07E
:1037000090681D12008CE493900061F08028900076
:10371000B0E0B428129000C6E090684712008CE434
:1037200093900061F0800F9000B0E0B446089000E4
:10373000A7E0900061F0900088E070089000C9E078
:1037400064046002800874039000C9F0D21F9000E6
:1037500065E0FE9000ADE0B50657900067E0FE9092
:1037600000CBE0B5064B900066E0FE9000D9E0B5D6
:10377000063F90006AE0FE900080E0B506339000BE
:1037800068E0FE9000BBE0B50627900069E0FE907F
:1037900000C9E0B5061B90006BE0FE9000E6E0B5C6
:1037A000060F90006CE0FE9000E7E06E70030239B7
:1037B0009490004BE0C39405500874029000FCF014
:1037C00080149000D9E0600874069000FCF0800638
:1037D000740A9000FCF0900080E0B4010674009040
:1037E0000080F0900080E0B4020674009000CBF0FE
:1037F000900080E0B4030674009000D8F09000CBF5
:10380000E0D394014027741B9000FEF074009006F2
:10381000C9F074009006CAF07400900095F0900012
:10382000ADE0B4020674019000ADF080339000ADBD
:10383000E0B4021A74009000FEF074009006C9F023
:1038400074009006CAF0741B900095F0801274000A
:103850009000FEF0741B9006C9F07400900095F083
:103860009000ADE06014741C900094F07400900619
:10387000CDF074009006CEF0800C7400900094F0AF
:10388000741C9006CDF09000E6E06014741990016D
:1038900000F074009006C1F074009006C2F0800C35
:1038A0007400900100F074199006C1F09000E7E0F8
:1038B0006014741A900101F074009006C5F0740051
:1038C0009006C6F0800C7400900101F0741A900606
:1038D000C5F09000D9E0701A74059006D1F0740616
:1038E0009006D5F074079006D9F074089006DDF0C4
:1038F000803074009006D1F074009006D2F074000D
:103900009006D5F074009006D6F074009006D9F0B9
:1039100074009006DAF074009006DDF074009006F2
:10392000DEF0D21F9000ADE0900065F09000D9E08D
:10393000900066F09000CBE0900067F09000BBE054
:10394000900068F09000C9E0900069F0900080E07D
:1039500090006AF09000E6E090006BF09000E7E0E5
:1039600090006CF0900080E0900886F09000C9E034
:10397000900888F09000BBE090088AF09000D9E0B1
:1039800090088BF09000ADE090088CF09000CBE0B8
:1039900090088DF09000E3E0B40117900021740FBF
:1039A000F0A374FFF0900023E4F0A3F07402900001
:1039B000E3F09000E3E0B40341900023E0FEA3E0D5
:1039C000FF900021E0FCA3E0FD1269F5741012697C
:1039D000AA7408120039EF90005EF0EF700674FFD1
:1039E00090005EF074009000E3F0900022E0900000
:1039F0005FF0900021E0900060F0900074E0900093
:103A000071F0900073E0900070F09000A2E0C39419
:103A10001E50569000A2E0F404241E900072F09014
:103A20000072E075F00A84FF7E008F73900072E0F0
:103A300075F00A84ADF07C008D74900070E0D39531
:103A400074400D900070E0C39574900070F0800F8A
:103A5000900070E0240AC39574900070F005739094
:103A60000071E02573900071F0900071E090003DCE
:103A7000F090003DE0241290003EF090003DE0D335
:103A80009448400B90003DE0C3944890003DF09076
:103A9000003EE0D39448400B90003EE0C394489031
:103AA000003EF0C22390003DE0D39424400D9000EE
:103AB0003DE0C3942490003DF0D223C22490003E08
:103AC000E0D39424400D90003EE0C3942490003E47
:103AD000F0D224900041E4F090003DE064236007C0
:103AE00090003DE0B4242090003DE0B42306740231
:103AF000900041F090003DE0B42406900041740134
:103B0000F090003D7401F0900042E4F090003EE03F
:103B10006423600790003EE0B4242090003EE0B4AF
:103B200023067402900042F090003EE0B424069018
:103B300000427401F090003E7401F0900074E0FEC9
:103B40009000D7E02E900044F0900044E0D39424FD
:103B5000400B900044E0C39424900044F090004453
:103B6000E0D39424400B900044E0C394249000449C
:103B7000F0900044E064126007900044E0B4240632
:103B8000900044E004F0900044E06411600790006D
:103B900044E0B42306900044E014F0900044E0D3E5
:103BA0009424400B900044E0C39424900044F0908F
:103BB0000044E0D39412400D900044E0C39412906E
:103BC0000045F0800A900044E02412900045F07512
:103BD00051129000BAE090003FF090003FE075F085
:103BE0001284AFF07E00EF4E700690003FE004F0CC
:103BF00090003FE00475F01284AFF07E00EF4E704D
:103C00000690003FE014F090003FE0B449069000B9
:103C10003F7401F090003FE0D39424400F90003FA8
:103C2000E0C3942490003FF0D21A8002C21A9000A0
:103C30003FE0D39412400D90003FE0C394129000F7
:103C400040F0800A90003FE02412900040F022C231
:103C500093C294C291C292C287C290E5B554EFF567
:103C6000B5E5B554DFF5B5C296C295C2A0C297C2FC
:103C7000A2C2A1E5B554BFF5B5E5B5547FF5B5E5EC
:103C8000B554FBF5B5C209755E469000BDE0700500
:103C9000756D028003756D037555007554009000B5
:103CA0000874FFF0A374DCF0C20EC21174C8900057
:103CB00035F074C8900039F0755300755200C20495
:103CC000754600E56FB40903756F007563009000D9
:103CD00017E4F0A3F0757010C20CC20DC203755743
:103CE0000075560090000AE4F0A3F090000CE4F098
:103CF000A3F0C22775590075580090007FE075F059
:103D000032A4FFAEF090001FEEF0A3EFF090006E33
:103D1000E4F090006FE4F0C222D217C216D218C2AB
:103D200019C21AC21B22755B00755A00AE5AAF5BEE
:103D30007402C39F74019E5003023DE490667912A1
:103D40000048E4939000731269DB0FBF00010EE09E
:103D5000FC906679120048ECFEE493FFEEC39F509E
:103D600026AE5AAF5B0FBF00010E90667912004875
:103D7000AE5AAF5BE493FC906679120048E49390EE
:103D800000731269DBECF0AE5AAF5B9066791200FB
:103D900048E4939000731269DBE0FC90667B1200AC
:103DA00048ECFCE493FDECD39D401990667B120037
:103DB00048E493FC906679120048E49390007312F3
:103DC00069DBECF0AE5AAF5B74022FFF50010E8E30
:103DD0005A8F5B785B740126F6500418E436F6407F
:103DE00003023D2C22755B00755A00AE5AAF5B741E
:103DF00033BE00039F5003023EB290677B1200481F
:103E0000E4939000731269DB0FBF00010EE0FC9099
:103E1000677B120048ECFEE493FFEEC39F5026AE92
:103E20005AAF5B0FBF00010E90677B120048AE5A7D
:103E3000AF5BE493FC90677B120048E493900073BF
:103E40001269DBECF0AE5AAF5B90677B120048E47E
:103E5000939000731269DBE0FC90677D120048ECE0
:103E6000FCE493FDECD39D401990677D120048E47B
:103E700093FC90677B120048E4939000731269DB17
:103E8000ECF0AE5AAF5B742D6F4E7006755B3375F8
:103E90005A00AE5AAF5B74022FFF50010E8E5A8F3C
:103EA0005B785B740126F6500418E436F640030292
:103EB0003DEB22755B00755A00AE5AAF5B7433BEA2
:103EC00000039F5003023F809067AE120048E493C6
:103ED0009000731269DB0FBF00010EE0FC9067AE2B
:103EE000120048ECFEE493FFEEC39F5026AE5AAF9B
:103EF0005B0FBF00010E9067AE120048AE5AAF5B79
:103F0000E493FC9067AE120048E49390007312694A
:103F1000DBECF0AE5AAF5B9067AE120048E49390D2
:103F200000731269DBE0FC9067B0120048ECFCE41F
:103F300093FDECD39D40199067B0120048E493FCC8
:103F40009067AE120048E4939000731269DBECF0C6
:103F5000AE5AAF5B742D6F4E7006755B33755A00A9
:103F6000AE5AAF5B74022FFF50010E8E5A8F5B78F2
:103F70005B740126F6500418E436F64003023EB99D
:103F800022755B00755A00AE5AAF5B7433BE0003F6
:103F90009F500302404E9067E1120048E493900066
:103FA000731269DB0FBF00010EE0FC9067E11200A5
:103FB00048ECFEE493FFEEC39F5026AE5AAF5B0F72
:103FC000BF00010E9067E1120048AE5AAF5BE49368
:103FD000FC9067E1120048E4939000731269DBECF7
:103FE000F0AE5AAF5B9067E1120048E49390007323
:103FF0001269DBE0FC9067E3120048ECFCE493FDFF
:10400000ECD39D40199067E3120048E493FC90675D
:10401000E1120048E4939000731269DBECF0AE5AB1
:10402000AF5B742D6F4E7006755B33755A00AE5AD8
:10403000AF5B74022FFF50010E8E5A8F5B785B745A
:104040000126F6500418E436F64003023F8722E5C5
:104050000C906218F828287302411575E700A23009
:10406000B34008E5B54408F5B58006E5B554F7F565
:10407000B575E71002411575E700A230B34008E5B9
:10408000B54402F5B58006E5B554FDF5B575E71004
:10409000024115A23092A2807CA23092A180767556
:1040A000E700A230B34008E5B54440F5B58006E529
:1040B000B554BFF5B575E710805B75E700A230B366
:1040C0004008E5B54480F5B58006E5B5547FF5B503
:1040D00075E7108040A2309287803AA2309290809B
:1040E0003475E700A230B34008E5B54410F5B5805B
:1040F00006E5B554EFF5B575E710801975E700A230
:1041000030B34008E5B54420F5B58006E5B554DF89
:05411000F5B575E71094
:1062180002405802405B02407702409302409902D4
:10622800409F0240BA0240D50240DB0240E10240F2
:01623800FC69
:104115002285F97385FA747E017F00E5741269AA18
:10412500E5732FFF50010E8E5A8F5BAC5CAD5DEFD2
:104135002DFDEE3CFC8C5C8D5DD293D294D291D258
:1041450092E55DF5FBE55CF5FCE55DF5E9E55CF51E
:10415500EAE55DF5EBE55CF5ECE55DF5EDE55CF5D2
:10416500EE2275A71085F97385FA747E017F00E547
:10417500741269AAE5732FFF50010E8E5A8F5B7E6C
:10418500017F769000F8E01269AAAC5AAD5BED2F7D
:10419500FFEC3EFE8E5C8F5DE55DF5FDE55CF5FEB5
:1041A500900062E4F075A7007412900047F0228534
:1041B500F97385FA747E017F00E5741269AAE573C7
:1041C5002FFF50010E8E5A8F5B900011E0FCA3E08B
:1041D500FDEF2DFDEE3CFC8C5C8D5DE55DF5FDE5B3
:1041E5005CF5FE220564229000BBE0B40353900009
:1041F500D9E0B4012EA2D8B34004C293C287A2D994
:10420500B34004C294C290A2DAB34008C291E5B5A6
:1042150054EFF5B5A2DBB34008C292E5B554DFF51E
:10422500B5801CA2D8B34002C293A2D9B34002C242
:1042350094A2DAB34002C291A2DBB34002C29280DB
:104245002EA2D8B34012C293C2919000D9E0600863
:10425500C287E5B554EFF5B5A2D9B34012C294C2F1
:10426500929000D9E06008C290E5B554DFF5B5A29B
:10427500DCB34030A29650067419900047F0A29521
:1042850050067419900047F0A2A0500674199000CA
:1042950047F0A29750067419900047F0C296C29550
:1042A500C2A0C29775D8402285A77275A710A2D85B
:1042B500B34002C287A2D9B34002C290A2DAB3408A
:1042C50006E5B554EFF5B5A2DBB34006E5B554DF19
:1042D500F5B5A2DCB340089000C7E0900062F07528
:1042E500D8408572A72290F800E4936406600280A6
:1042F500FE75B50075840175A70075FF8075EF061D
:10430500900043E4F075C91075A70F75A1C775A78F
:104315000075D90075CE0C75A70F75F1FE75F2FF06
:1043250075F30775F47875A4BA75A5FF75A60775B5
:10433500AE0075AFFF75D48175D5FF75D6FF75D7FE
:10434500FF75A70075A20175A14775F80975D80015
:1043550075D90475DA0975DB0975DC0975DD09752B
:10436500DE0975D84075A71075D80075D90475DABA
:104375000975DB0975DC0975DD0975DE0975D84038
:1043850075A70075E60875E71075BC0175BE04755F
:10439500BD6C75BE0775BDA075BE0875BD0175BC44
:1043A5000075BB1875BC2075BA0875E88075D11302
:1043B50075A70F75E10575E20075C740123C4F758D
:1043C5009700759780740A12698A7597C0E59754A6
:1043D50020700280F8758F0275A700D2AF7598001E
:1043E50075A90C75A70F75AB4375ADFB75AC1E753F
:1043F500A71075C91875CA0075CB0075C80475A7CF
:1044050000758912758E04758C00758A00C2A9D253
:104415008C758D00758B00D2ABD28E75B62075D993
:1044250044C299C22674C8F5097508001200F875CA
:10443500A70FE5FB900051F0E5FA900052F0E5F981
:10444500900053F075A70090F800E493F527120249
:1044550017900886E0D3940340067400900886F010
:1044650074019000BCF0900886E0906239F8282825
:1044750073802A802875A70F75F30F75A700A2A36F
:10448500400674029000BCF0801375A70F75F317F2
:0D44950075A700A2A4400674029000BCF0C0
:0C62390002447602447802447A02448F4A
:1044A2009000BCE0B4022AC2251205B67402900044
:1044B200BCF0900886E0906245F82828738010804E
:0F44C2000E74009000CBF0800674009000D8F0CC
:0C6245000244BF0244C10244C30244CB27
:1044D1008028D2251204D574019000BCF090088682
:1044E100E0906251F82828738010800E74009000CB
:0A44F100CBF0800674009000D8F0B4
:0C6251000244E90244EB0244ED0244F573
:1044FB001233109000C6E07006740A9000C6F0905C
:10450B0000A7E0700674E39000A7F09000ADE00404
:10451B00900065F012358390F807E493900058F003
:10452B00900058E0440A900058F0900058E054FE78
:10453B00900058F07406900049F0740190004AF016
:10454B0090F802E49390004BF0740390004CF074DD
:10455B000590004DF0741490004EF0740690004FCF
:10456B00F090004BE0B40406740490004FF0900000
:10457B004BE0B40506740590004FF07406900050A4
:10458B00F090F804E493900054F07400900055F010
:10459B0090F805E493900056F090F806E4939000A1
:1045AB0057F074FF900059F0123D2690004BE0B489
:1045BB000505123EB3801190004BE0D394054005E6
:1045CB00123DE58003123F819000E2E090005EF027
:1045DB00900099E090005FF090009AE0900060F0FE
:1045EB00A2B6B39205A2B3B39206A2A4B3921DA234
:1045FB00A3B3921E90005AE4F0756F00743A9007C3
:10460B0073F074FD900774F090005BE4F0756E012D
:10461B00900047E4F09000BDE0B40106741A9000DE
:10462B0047F0C21C756300C20AD20BC2037571003E
:10463B00C21F12009E755F00756B0075610075657A
:10464B0032756600756700756800756900756A00DC
:10465B00900017E4F0A3F0756C00D2B2D2A4D2B0E4
:10466B00D2B1D2A3D2A7D2A6D2A5D2B790007FE067
:10467B00D394FA400674FA90007FF07E017F00908D
:10468B000060E01269AA90005FE02FFF50010E90CE
:10469B000021EEF0A3EFF0EFD394FFEE940F400761
:1046AB00900021E4F0A3F090005EE0700674FF90A0
:1046BB00005EF09000BDE07005756D028003756DB6
:1046CB00039000BEE0D39401400674009000BEF04E
:1046DB009000C4E0C3940A5006740A9000C4F09092
:1046EB0000CEE0700674019000CEF09000CEE0B4E6
:1046FB00FF0674FE9000CEF09000D5E0D394FE4000
:10470B000674FE9000D5F09000FBE0D394024006B7
:10471B0074019000FBF0900111E0D39401400674FA
:10472B0001900111F074019000DBF074019000DC3A
:10473B00F074009000E3F074009000FFF0740090B0
:10474B000103F074299006B9F0742A9006BDF0D2DB
:10475B009C9000AEE0D39404400674049000AEF03D
:10476B009000E0E0D39404400674049000E0F0E580
:10477B0070D3941040037570109006BAE0D3940C6C
:10478B00400674009006BAF09006BEE0D3940C403D
:10479B000674009006BEF09006C2E0D3940C40065F
:1047AB0074009006C2F09006C6E0D3940C400674D9
:1047BB00009006C6F09006CAE0D3940C4006740035
:1047CB009006CAF09006CEE0D3940C40067400908D
:1047DB0006CEF09006D2E0D3940C400674009006FF
:1047EB00D2F09006D6E0D3940C400674009006D617
:1047FB00F09006DAE0D3940C400674009006DAF0E1
:10480B009006DEE0D3940C400674009006DEF0D2E6
:10481B00EC75CF01A298B34005C298120697E54DEF
:10482B006006A299B3B340028005C299120B78E5DA
:10483B004E64016005E54EB4040280D5C28E7E1035
:10484B007F00E5641269AAE58D75F010A4FDACF04C
:10485B00EF2DFDEE3CFCE58B75F01084FF7E00ED3B
:10486B002FFFEC3EFE8E548F55D28E9000A0E06051
:10487B00099000A0E0C3943D4002805C90001912A7
:10488B0069B8900019E0FEA3E0FF90001BE0FCA3C9
:10489B00E0FDEFB50542EEB5043EB214A204B34001
:1048AB001975E700A214B34008E5B54404F5B580CB
:1048BB0006E5B554FBF5B575E71090001BE0FEA3BC
:1048CB00E0FF90001DE0FCA3E0FDEF2DFDEE3CFCB6
:1048DB0090001BECF0A3EDF09000ADE060099000B0
:1048EB00ADE0C394034003024996122745A204B3DB
:1048FB00500990005AE0C3941C4002800690009728
:10490B00E0F545E54575F002A4FFAEF090087BEEAF
:10491B00F0A3EFF0900084E0C395614007E55FC31F
:10492B009560500790087BE4F0A3F075E700AE2E7E
:10493B00AF2F90087BE0FCA3E0FDEFD39DEE9C40F6
:10494B0020E5B5547FF5B59000ADE0B402099000B9
:10495B00CBE0C3940240028006E5B54440F5B58038
:10496B002790005AE0C3942A501EE5B54480F5B554
:10497B009000ADE0B402099000CBE0C3940240027A
:10498B008006E5B554BFF5B575E7109000ADE0B402
:10499B00032A12286075E700AE2EAF2F90087BE03C
:1049AB00FCA3E0FDEFD39DEE9C4008E5B54480F5FC
:1049BB00B58006E5B5547FF5B575E710900088E036
:1049CB006009A2B3300601B3B340028056A2B330E4
:1049DB000601B3404EA2B3300801B34039A21740D1
:1049EB003090006DE0D3955E402590006FE0701322
:1049FB0090006EE0B4010690006F7401F090006EB1
:104A0B00E004F0A216B3400590006EE4F0D216D28B
:104A1B0017A208B39206A208B330B301B34004A2A5
:104A2B00089206A2B6300501B350030250DCA2B6C1
:104A3B00300501B350030250DCA2B6300701B3506E
:104A4B0003024F88756E009000A0E0B43D1975E726
:104A5B0000A207B34008E5B554FBF5B58006E5B5F4
:104A6B004404F5B575E710055EA209B3B35013AE58
:104A7B0054AF55900008E0FCA3E0FDEDC39FEC9E06
:104A8B004003024C57E56DB4032EA227B34022E539
:104A9B005EB42303756D01E55EC39423500690004D
:104AAB00477401F0E55ED3942340067402900047EF
:104ABB00F0755E01D2278062E56DB4020A756D0157
:104ACB00755E23C216C218E55EB42305755E0180C0
:104ADB0049900047E07034E55EC394235006900084
:104AEB00477401F0E55ED3942340067402900047AF
:104AFB00F0E55EC394235002D21CE55ED3942340B1
:104B0B0002D21CC296C295C2A0C2979000BDE0B45F
:104B1B000105123C4F8003755E01AE56AF57AC5486
:104B2B00AD55EF2DFDEE3CFC74028C068D0712008B
:104B3B00398E568F579000A0E060099000A0E0C31B
:104B4B00943D40028049900019E0FEA3E0FF9000E5
:104B5B00A0E08E048F05FF12699A74018C068D07F5
:104B6B0012003990001DEEF0A3EFF090001DE0F85D
:104B7B00A3E090001BC8F0A3C8F0900019E4F0A3C9
:104B8B00F0C21475E700E5B554FBF5B575E710A257
:104B9B00A4B34002C21DA2A3B34002C21EA21CB307
:104BAB004002C21CB21990006FE0B40111A216B3FF
:104BBB004004D2198002C219740290006FF0900069
:104BCB006FE0C394025006A204B3B3400280067494
:104BDB000290006FF09000C9E0640460079000BB86
:104BEB00E0B40362900088E0600690006FE0700212
:104BFB00800DA218301601B3400590006EE4F090C2
:104C0B0000BDE064016006A222B3B3501790008888
:104C1B00E06009A216301801B3B340028006740598
:104C2B00900047F0B218A217B3401BA216B3400472
:104C3B00D2188002C2189000BDE0700690006FE0A1
:104C4B0070028002D222C216C217803AAE56AF57FC
:104C5B00AC54AD55EF2DFDEE3CFC74018C068D076D
:104C6B001200398E568F57E56DC39402500DAC541C
:104C7B00AD557488C39D74139C40028009123C4F40
:104C8B007406900047F0E55EB4231274039000475E
:104C9B00F0D21C9000BDE0B40103123C4FAE58AFF4
:104CAB0059AC54AD55EF2DFDEE3CFC8C588D59AEE7
:104CBB0054AF55EFD39DEE9C401190000FE0FAA33B
:104CCB00E0FBEBC394E8EA94034002800690000FEC
:104CDB001269B890000CE0FEA3E0FFAC54AD55EFA9
:104CEB002DFDEE3CFC90000CECF0A3EDF09000BD24
:104CFB00E0B40118AE54AF5574051269AA740112D1
:104D0B000039900008EEF0A3EFF08011AE54AF55D0
:104D1B0074021269AA900008EEF0A3EFF0C28E7530
:104D2B008D00758B00756400755501755400D28E1E
:104D3B00E55E240875F00984AFF07E00EF4E60034A
:104D4B00024DD0E56D6013AE56AF5774091269AAC8
:104D5B0090000AEEF0A3EFF0800F90000CE0F8A3A8
:104D6B00E090000AC8F0A3C8F090000AE0FEA3E0B0
:104D7B00FFEF4E600B7C797DAB1268988E528F5390
:104D8B0090000CE4F0A3F0AE52AF537428BE0003B6
:104D9B009F5010E5632FFF50010E74011200398EE6
:104DAB00528F538553639000C4E0A852B8000DD3C3
:104DBB0095534008E553900046F080099000C4E0FD
:104DCB0014900046F09000BBE0B4030890003FE065
:104DDB00655E6002800EA219301A01B34004D21B2B
:104DEB008002C21BE55E640B6005E55EB41D099095
:104DFB0000ADE06003122411900044E0655E600793
:104E0B00900045E0B55E03756F00A20AB35006A291
:104E1B0009B3B34003024EC8900079E0B40173901C
:104E2B0000FBE0B40214120D19900063E075F0BEA4
:104E3B00A4FFAEF08E5C8F5D8056E56775F00A843B
:104E4B00FF7E00900573120048E0F55B755A00AECB
:104E5B005AAF5B90009EE01269AA74648E048F05B2
:104E6B00FF12699A8C5C8D5DE55D90000EF0AE5A79
:104E7B00AF5B900077E01269AA74648E048F05FF14
:104E8B0012699A74BE8C068D071269AA8E5C8F5DAF
:104E9B008017900077E075F0BEA4FFAEF08E5C8FAC
:104EAB005D90009EE090000EF0E561C394CC50063F
:104EBB00E55D455C70028003124116D20AE56DB4C4
:104ECB000106E55E640B600280189000C9E0B40433
:104EDB000575700380097570019000487401F075B9
:104EEB006D00E56D6003024F839000C0E0600D9094
:104EFB000062E0A852B8000695534002803890003B
:104F0B00C0E0B4021790003DE0655E600790003E84
:104F1B00E0B55E03757003756C00800CC201756C97
:104F2B0000900017E4F0A3F0900062E060067409B3
:104F3B00900047F0804290003DE0655E6007900076
:104F4B003EE0B55E339000C9E0B4040FA222B3403B
:104F5B0005757001800375700380037570019000F7
:104F6B003DE0B55E069000487401F090003EE0B560
:104F7B005E067402900048F0A207B39205A207B335
:104F8B0030B601B350030250DC756E019000A0E007
:104F9B00B43D1975E700A207B34008E5B54404F525
:104FAB00B58006E5B554FBF5B575E710A2264005AF
:104FBB0075FFA0D22675E700E5B54401F5B575E799
:104FCB0010741C90005AF0A2079205E55ED3944A28
:104FDB004014D209E55ED3946D400B7404900047E6
:104FEB00F0D21C755E469000C8E0B40107E56AC3B9
:104FFB00941440028009123C4F7413900047F0E563
:10500B006AC394415009740E900047F0123C4F90C4
:10501B00004FE0FE90004BE0C39E400990004BE038
:10502B00D39408400974FB900047F0123C4F90005A
:10503B0054E06015900054E0FE90004EE06E600965
:10504B0074FE900047F0123C4F900886E06006908B
:10505B0000F8E06002807A74019000BCF090088642
:10506B00E090625DF828287380188016A2A3400692
:10507B0074029000BCF0800AA2A440067402900057
:02508B00BCF077
:0C625D000250730250750250770250830B
:10508D009000BCE0B40105A225B340028019D225E1
:10509D00123C4F1204D574019000BCF0123310D2A3
:1050AD001F741B900047F09000BCE0B40206A225CF
:1050BD00B3B340028019C225123C4F1205B67402DB
:1050CD009000BCF0123310D21F741B900047F0A259
:1050DD001CB34008C296C295C2A0C2979000F8E0DA
:1050ED00600CAE52AF537414BE00059F4002803762
:1050FD00900080E0906269F8282873802A8028A2A9
:10510D00A3B35005A21EB340028005124167D21E03
:10511D008015A2A4B35005A21DB340028005124113
:07512D0067D21D8002800023
:1062690002510802510A02510C02511F0251320215
:0262790051349E
:10513400A20CB3B3500890003FE0655E60030253D5
:105144006DA202B35006A201B3B3400302536990A7
:1051540000BBE0B40302800302532890006FE0B464
:105164000202800302530FA21BB3500302523C12EB
:10517400347090010CE0601F900015E0FEA3E0FF86
:10518400900104E01269AA74C88E048F05FF1269A5
:105194009A8C5C8D5D800A900015E0F55CA3E0F5C7
:1051A4005DAE5CAF5D745E1269AA74058E048F05F2
:1051B400FF12699AAE5AAF5BED2FFFEC3EFE8E5C98
:1051C4008F5DE55DF5FBE55CF5FCD293A203B3408E
:1051D40002D2879000D9E0B4025B12349D90010C96
:1051E400E0D39404401BAE2CAF2D900108E012696B
:1051F400AA74C88E048F05FF12699A8C5C8D5D8039
:1052040006852C5C852D5DAE5CAF5D745E1269AA6B
:1052140074058E048F05FF12699AAE5AAF5BED2FA9
:10522400FFEC3EFE8E5C8F5DE55DF5FBE55CF5FC19
:1052340075A700D28702530D12347090010CE0D38D
:105244009403401F900015E0FEA3E0FF900106E0E8
:105254001269AA74C88E048F05FF12699A8C5C8D3A
:105264005D800A900015E0F55CA3E0F55DAE5CAFEF
:105274005D745E1269AA74058E048F05FF12699A23
:10528400AE5AAF5BED2FFFEC3EFE8E5C8F5DE55DAD
:10529400F5EBE55CF5ECD291A203B34006E5B54429
:1052A40010F5B59000D9E0B4025F12349D90010C62
:1052B400E0D39406401BAE2CAF2D90010AE0126996
:1052C400AA74C88E048F05FF12699A8C5C8D5D8068
:1052D40006852C5C852D5DAE5CAF5D745E1269AA9B
:1052E40074058E048F05FF12699AAE5AAF5BED2FD9
:1052F400FFEC3EFE8E5C8F5DE55DF5EBE55CF5EC69
:1053040075A700E5B54410F5B58017123470E55D56
:10531400F5FBE55CF5FCE55DF5EBE55CF5ECD293BE
:10532400D2918041123470E55DF5FBE55CF5FCD269
:1053340093D291A203B34008D287E5B54410F5B5E2
:105344009000D9E0B4021E12349DE55DF5FBE55CE6
:10535400F5FCE55DF5EBE55CF5EC75A700D287E5BA
:10536400B54410F5B5C20CD20DA20DB3B3500890DC
:105374000040E0655E60030255A9A202B35006A294
:1053840001B3B340030255A59000BBE0B40302800F
:105394000302556490006FE0B40202800302554B8F
:1053A400A21BB3500302547812347090010CE0D362
:1053B4009401401F900015E0FEA3E0FF900105E07A
:1053C4001269AA74C88E048F05FF12699A8C5C8DC9
:1053D4005D800A900015E0F55CA3E0F55DAE5CAF7E
:1053E4005D745E1269AA74058E048F05FF12699AB2
:1053F400AE5AAF5BED2FFFEC3EFE8E5C8F5DE55D3C
:10540400F5E9E55CF5EAD294A203B34002D29090A8
:1054140000D9E0B4025B12349D90010CE0D39405F2
:10542400401BAE2CAF2D900109E01269AA74C88EFE
:10543400048F05FF12699A8C5C8D5D8006852C5C57
:10544400852D5DAE5CAF5D745E1269AA74058E0431
:105454008F05FF12699AAE5AAF5BED2FFFEC3EFE4B
:105464008E5C8F5DE55DF5E9E55CF5EA75A700D234
:105474009002554912347090010CE0D39403401FFC
:10548400900015E0FEA3E0FF900107E01269AA7402
:10549400C88E048F05FF12699A8C5C8D5D800A901A
:1054A4000015E0F55CA3E0F55DAE5CAF5D745E12E3
:1054B40069AA74058E048F05FF12699AAE5AAF5B10
:1054C400ED2FFFEC3EFE8E5C8F5DE55DF5EDE55C5A
:1054D400F5EED292A203B34006E5B54420F5B590AB
:1054E40000D9E0B4025F12349D90010CE0D394071C
:1054F400401BAE2CAF2D90010BE01269AA74C88E2C
:10550400048F05FF12699A8C5C8D5D8006852C5C86
:10551400852D5DAE5CAF5D745E1269AA74058E0460
:105524008F05FF12699AAE5AAF5BED2FFFEC3EFE7A
:105534008E5C8F5DE55DF5EDE55CF5EE75A700E548
:10554400B54420F5B58017123470E55DF5E9E55CE6
:10555400F5EAE55DF5EDE55CF5EED294D292804195
:10556400123470E55DF5E9E55CF5EAD294D292A2D5
:1055740003B34008D290E5B54420F5B59000D9E0D6
:10558400B4021E12349DE55DF5E9E55CF5EAE55DDE
:10559400F5EDE55CF5EE75A700D290E5B54420F590
:1055A400B5D20CC20DE57090627BF8282873025ABC
:0555B4000D9000E0E095
:06627B000255B20255B508
:1055B9009062F6F8282873121DB38012121DB38069
:0E55C9000D121E3D8008121EE98003121EE91D
:0F62F6000255C00255C50255CA0255CF0255D4F4
:1055D700757002025A0D12201512212C12244690C2
:1055E7000873E0FEA3E0FF740A1269AA90000AE0BC
:1055F700FCA3E0FD74098F02FF12699A8D078C03E3
:105607008E048A058B06126898900877EEF0A3EF50
:10561700F09000C9E0B401087478BE00059F40020D
:10562700800D7478900877F8E4F0E8A3F0801B9079
:105637000877E0FEA3E0FF74F0BE00039F500B74F1
:10564700F0900877F8E4F0E8A3F0E53670037536D4
:1056570001900877E0FEA3E0FFE5362FFF50010E2B
:0F566700900877EEF0A3EFF0757003900048E025
:036281000255DDE6
:10567600906305F82828738010A22F400375700ADE
:095686008007A22F400375700B90
:0963050002567D02567F02568803
:10568F00025A0D9006BAE060077401F50812256DF5
:10569F009000F9E0B401149000FAE0A852B80004A9
:1056AF0095535007E55FC3956040028009741590CC
:1056BF000047F00257469000AEE0D39402403F906F
:1056CF000082E02403A852B80004955350099000BB
:1056DF0084E0D3956150028008D20274089000478D
:1056EF00F0900082E0A852B80005D39553500B906C
:1056FF000084E02403C395615002C20280399000F8
:10570F0082E02403A852B8000495535007E55FC305
:10571F00956040028008D2027408900047F0900014
:10572F0082E0A852B80005D395535009E560240FC5
:10573F00C3955F5002C2029000C8E07007E56AC3CC
:10574F00941440028002D2029000BDE0B40102D254
:10575F0002A2024005757004800A75701090001740
:0B576F00E4F0A3F0025A0D9000AEE041
:066284000256920257765B
:10577A0090630EF8282873120E038012120E03800B
:0E578A000D120FB1800812106380031210631D
:0F630E0002578102578602578B0257900257950C
:105798009006BEE060077402F50812256D75700565
:1057A800025A0D1211A37570069006C2E0600774C4
:1057B80003F50812256D9006C6E060077404F50825
:1057C80012256D025A0D90000EE06006A204B3B3D4
:1057D8004002801D90000EE02529FFAE2850010EE2
:1057E8008E288F29E55ED39412500690000EE0149F
:1057F800F01213E97570079006CAE060077405F5A2
:105808000812256D9006CEE060077406F50812258B
:105818006D025A0D9000FBE0B40203120D911218AC
:10582800197570089006D2E060077407F50812250C
:105838006D9006D6E060077408F50812256D025AC7
:105848000D121BD5A20CB35005A20DB34002800463
:10585800D20CD20D7570109006DAE060077409F565
:105868000812256D9006DEE06007740AF508122517
:105878006D025A0D025A0D900037E0C39446500A43
:10588800C296C2A07446900037F0900041E0B4017F
:105898001DE536240AF536900877E0FEA3E0FF748C
:1058A8000A2FFF50010E900877EEF0A3EFF090005A
:1058B80041E0B4021DE5362414F536900877E0FE81
:1058C800A3E0FF74142FFF50010E900877EEF0A3A9
:1058D800EFF085365B755A0090003DE0F5731234A1
:1058E800E8E55D900037F0900004E55AF0A3E55B29
:1058F800F0E573900038F0C20F900877E0F55AA3EE
:10590800E0F55B90003DE0F5731234E8E55D90004A
:1059180035F0900000E55AF0A3E55BF0E5739000E0
:1059280036F0A2009210900041E06002B210C20E60
:10593800757003025A0D90003BE0C39446501390D3
:1059480000C9E0B40102C296C295C297744690009D
:105958003BF0900042E0B4011DE536240AF536908C
:105968000877E0FEA3E0FF740A2FFF50010E9008AD
:1059780077EEF0A3EFF0900042E0B4021DE5362484
:1059880014F536900877E0FEA3E0FF74142FFF505B
:10599800010E900877EEF0A3EFF085365B755A009C
:1059A80090003EE0F5731234E8E55D90003BF0901E
:1059B8000006E55AF0A3E55BF0E57390003CF0C201
:1059C80012900877E0F55AA3E0F55B90003EE0F509
:1059D800731234E8E55D900039F0900002E55AF062
:1059E800A3E55BF0E57390003AF0A20092139000F3
:1059F80042E06002B213C21175700380088006800D
:055A0800048002800093
:10628A000257AB0257CE02581C02584902587C02E8
:10629A00587F02593E025A05025A07025A09025AFF
:0462AA000B025A0D7C
:105A0D00900035E0B55E028003025AEAA20E4072A4
:105A1D00900000E0FEA3E0FFEF4E6021AE56AF57C1
:105A2D00900000E0FCA3E0FD120003740A8E048FC9
:105A3D0005FF12699A900000ECF0A3EDF09000368E
:105A4D00E0601A900000E0FEA3E0FFAC56AD57EF0A
:105A5D002DFDEE3CFC900000ECF0A3EDF090003637
:105A6D00E0D39401401A900000E0FEA3E0FFAC5695
:105A7D00AD57EF2DFDEE3CFC900000ECF0A3EDF0EA
:105A8D00D20EAE54AF55900000E0FCA3E0FDEFC385
:105A9D009DEE9C40481241B49000C9E09062AEF872
:105AAD002828738030D296802CD2968028D296D218
:105ABD00A08022A2104010A223301801B34004D2BE
:105ACD00A08002D296800EA223301801B34004D2DA
:055ADD00968002D2A03A
:0F62AE00025AB0025AB2025AB6025ABA025AC083
:105AE200C20E74C8900035F0A20EB3B350079000F6
:105AF20035E0B55E0280481241B49000C9E0906280
:105B0200BDF82828738030D296802CD2968028D275
:105B120096D2A08022A2104010A223301801B340D6
:105B220004D2A08002D296800EA223301801B34084
:075B320004D2968002D2A00C
:0F62BD00025B07025B09025B0D025B11025B17BC
:105B390074C8900035F0C20E900037E0B55E02805F
:105B490003025BE2A20F4072900004E0FEA3E0FFB3
:105B5900EF4E6021AE56AF57900004E0FCA3E0FD84
:105B6900120003740A8E048F05FF12699A900004CB
:105B7900ECF0A3EDF0900038E0601A900004E0FE2C
:105B8900A3E0FFAC56AD57EF2DFDEE3CFC900004B1
:105B9900ECF0A3EDF0900038E0D39401401A9000A6
:105BA90004E0FEA3E0FFAC56AD57EF2DFDEE3CFC43
:105BB900900004ECF0A3EDF0D20FAE54AF55900075
:105BC90004E0FCA3E0FDEFC39DEE9C400CC296C22D
:105BD900A07446900037F0C20FA20FB3B3500790DC
:105BE9000037E0B55E02800CC296C2A074469000F0
:105BF90037F0C20F900039E0B55E028003025CDA2B
:105C0900A2114072900002E0FEA3E0FFEF4E602176
:105C1900AE56AF57900002E0FCA3E0FD12000374FA
:105C29000A8E048F05FF12699A900002ECF0A3ED29
:105C3900F090003AE0601A900002E0FEA3E0FFACA9
:105C490056AD57EF2DFDEE3CFC900002ECF0A3EDB4
:105C5900F090003AE0D39401401A900002E0FEA3CC
:105C6900E0FFAC56AD57EF2DFDEE3CFC900002EC89
:105C7900F0A3EDF0D211AE54AF55900002E0FCA3B1
:105C8900E0FDEFC39DEE9C40481241B49000C9E08D
:105C99009062CCF82828738030D296802CD29580D7
:105CA90028D295D2978022A2134010A2243018013D
:105CB900B34004D2978002D295800EA224301801F5
:095CC900B34004D2958002D29789
:0F62CC00025CA0025CA2025CA6025CAA025CB0AB
:105CD200C21174C8900039F0A211B3B350079000FA
:105CE20039E0B55E0280481241B49000C9E090628A
:105CF200DBF82828738030D296802CD2958028D267
:105D020095D2978022A2134010A224301801B340EA
:105D120004D2978002D295800EA224301801B3409B
:075D220004D2958002D29724
:0F62DB00025CF7025CF9025CFD025D01025D07E7
:105D290074C8900039F0C21190003BE0B55E028062
:105D390003025DDBA2124072900006E0FEA3E0FFC1
:105D4900EF4E6021AE56AF57900006E0FCA3E0FD90
:105D5900120003740A8E048F05FF12699A900006D7
:105D6900ECF0A3EDF090003CE0601A900006E0FE34
:105D7900A3E0FFAC56AD57EF2DFDEE3CFC900006BD
:105D8900ECF0A3EDF090003CE0D39401401A9000B0
:105D990006E0FEA3E0FFAC56AD57EF2DFDEE3CFC4F
:105DA900900006ECF0A3EDF0D212AE54AF5590007E
:105DB90006E0FCA3E0FDEFC39DEE9C40159000C9F1
:105DC900E0B40102C296C295C297744690003BF0B6
:105DD900C212A212B3B3500790003BE0B55E028035
:105DE900159000C9E0B40102C296C295C2977446E3
:105DF90090003BF0C2129000CBE0B4020280030293
:105E09005F3390005CE0D39566506490005CE0F4E9
:105E1900042566FE9000CEE08E00F5F0E884FF7E52
:105E2900008F73EFC39410500CEF8573F0A4FDAC91
:105E3900F08D7380037573FF90005CE0D395734018
:105E49000B90005CE0C39573F57180037571009048
:105E590000E9E0D3957140069000E9E0F571900002
:105E6900EAE0C3957150069000EAE0F571807190FF
:105E7900005CE0C39566FE9000CEE08E00F5F0E888
:105E890084FF7E008F73EFC39410500CEF8573F07D
:105E9900A4FDACF08D7380037573FF85735B755A30
:105EA9000090005CE0255BFFAE5A50010E8E5A8FC0
:105EB9005B74FFBE0009D39F4005855B7180037544
:105EC90071FF9000E9E0D3957140069000E9E0F593
:105ED900719000EAE0C3957150069000EAE0F5710F
:105EE900A204B3B3500D90005DE0FE9000D6E0D35C
:105EF9009E500280147407900047F075E700E5B5DD
:105F090054BFF5B575E710802175A71075E700E551
:105F1900CDC395714008E5B554BFF5B58006E5B523
:105F29004440F5B575E71075A7009000E6E0604EAE
:105F39009000F0E0A852B80004955350179000EF74
:105F4900E0A852B8000ED3955340099000F1E0D370
:105F590095614002801575A710E5CDC394BF400433
:105F6900C2A28002D2A275A700801375A710E5CD41
:105F7900C394404004C2A28002D2A275A700900037
:105F8900E7E0604E9000F3E0A852B8000495535042
:105F9900179000F2E0A852B8000ED395534009902B
:105FA90000F4E0D395614002801575A710E5CDC3D3
:105FB90094BF4004C2A18002D2A175A700801375C5
:105FC900A710E5CDC394404004C2A18002D2A175B7
:105FD900A700E56FC39409500AA2EDB34005C2EDCD
:105FE900122A07AE54AF557498C39F743A9E400C59
:105FF90090005BE0C3945A4003026215A209B340C2
:1060090009123C4F7406900047F0A20BB3500EE5FD
:1060190061D394334007E561C394CC4002804A9030
:1060290000FBE0B40214120D19900063E075F05002
:10603900A4FFAEF08E5C8F5D800F900077E075F065
:1060490050A4FFAEF08E5C8F5DE55D455C601AA2E1
:1060590026400575FFA0D226E5B54401F5B5741CA7
:1060690090005AF0124116D20B90005BE0D39401D4
:106079004007E561C3941A40028002C20B9006BA38
:10608900E060077401F50812256D9006BEE060070F
:106099007402F50812256D9006C2E060077403F5D5
:1060A9000812256D9006C6E060077404F5081225EC
:1060B9006D9006CAE060077405F50812256D900613
:1060C900CEE060077406F50812256D9006D2E060EF
:1060D900077407F50812256D9006D6E06007740865
:1060E900F50812256D9006DAE060077409F50812C3
:1060F900256D9006DEE06007740AF50812256D909B
:10610900005BE0C3945A5026E56FB4090990005B1F
:10611900E004F0756F0090005BE0B45A0FA22640CE
:106129000575FFA0D226E5B54401F5B5803BE56FBD
:10613900B40903756F00755500755400758D0075A8
:106149008B0075640090005AE0C3942A50089000AF
:106159005AE004F08006742A90005AF090005AE040
:10616900B42A06E5B554FEF5B590005BE0D3940179
:106179004007E56AC3944140028009740E900047C4
:10618900F0123C4F900886E060069000F8E060024B
:10619900807A74019000BCF0900886E09062EAF879
:1061A90028287380188016A2A3400674029000BCA8
:0D61B900F0800AA2A4400674029000BCF021
:0C62EA000261AC0261AE0261B00261BC56
:1061C6009000BCE0B40105A225B340028019D22597
:1061D600123C4F1204D574019000BCF0123310D259
:1061E6001F741B900047F09000BCE0B40206A22585
:1061F600B3B340028019C225123C4F1205B6740291
:106206009000BCF0123310D21F741B900047F002AE
:02621600481C22
:10631D000000010001400160018001A001C001E009
:10632D0002000300039603B603D603F40400050030
:10633D000512052405360548055A056C057E0590A0
:10634D0005A805C005DE0600061406280646066EDD
:10635D0006AE05CF00FF013F015F017F019F01BF29
:10636D0001DF01FF02FF039503B503D503F303FF1F
:10637D0004FF05110523053505470559056B057DF9
:10638D00058F05A705BF05CE05F1061306270645A2
:10639D00066D06AD06ED05DD0FAA0FA50F9F0F9A31
:1063AD000F940F8D0F870F800F780F710F680F608F
:1063BD000F570F4E0F450F3B0F300F250F1A0F0EB6
:1063CD000F020EF50EE80EDB0ECC0EBE0EAE0E9FBE
:1063DD000E8E0E7D0E6C0E5A0E470E340E200E0CC8
:1063ED000DF70DE20DCB0DB50D9D0D850D6D0D54FC
:1063FD000D3A0D200D050CE90CCE0CB10C940C765C
:10640D000C580C3A0C1B0BFB0BDB0BBB0B9A0B79D3
:10641D000B570B350B130AF10ACE0AAB0A870A6428
:10642D000A400A1C09F809D409B0098C0967094307
:10643D00091F08FB08D608B2088E086A084608230B
:10644D0007FF07DC07B9079607730751072F070DDD
:10645D0006EC06CA06AA068906690649062A060A30
:10646D0005EC05CD05B0059205750558053C0520D3
:10647D00050504EA04CF04B5049C048204690451A3
:10648D0004390422040B03F403DE03C803B2039D95
:10649D00038903750361034D033B032803160304AE
:1064AD0002F202E102D102C002B002A00291028208
:1064BD000273026502570249023C022F02220216A4
:1064CD00020901FD01F201E601DB01D001C601BBAC
:1064DD0001B101A7019D0194018B01820179017028
:1064ED000168016001580150014801410139013233
:1064FD00012B0125011E01180111010B010500FFE2
:10650D0000FA0FA60FA00F990F920F8B0F840F7C1F
:10651D000F740F6B0F620F580F4E0F430F380F2C68
:10652D000F1F0F120F050EF70EE80ED80EC80EB77F
:10653D000EA50E930E800E6C0E580E420E2C0E15DF
:10654D000DFD0DE40DCB0DB10D950D790D5D0D3FCF
:10655D000D200D010CE10CC00C9E0C7C0C590C3562
:10656D000C100BEA0BC40B9E0B760B4F0B260AFD82
:10657D000AD40AAA0A800A550A2A09FF09D409A8C9
:10658D00097C0950092508F908CD08A10875084AA4
:10659D00081E07F307C8079D07730749072006F76D
:1065AD0006CE06A6067E06570630060A05E405BF8A
:1065BD00059B057705540532051004EF04CE04AE96
:1065CD00048F047104530435041903FD03E203C75A
:1065DD0003AD0394037B0363034B0334031E0308D2
:1065ED0002F302DE02CA02B602A30291027F026D1D
:1065FD00025C024C023C022C021D020E020001F252
:10660D0001E401D701CA01BE01B101A6019A018FB2
:10661D000185017A01700166015D0153014A014155
:10662D00013901310129012101190112010B010467
:10663D0000FD00F700F000EA00E400DE00D900D311
:10664D0000CE00C900C400BF00BA00B500B100AD56
:10665D0000A800A400A0009C009900950091008E58
:0C666D00008A008700840081007E007B12
:10009E0075470090087DE4F0A3F0753100753000CF
:1000AE00754D00754E00C22AD22C900886E0600273
:1000BE00D21F74FE90087FF8E4F0E8A3F074FE906F
:1000CE000883F8E4F0E8A3F074FE900881F8E4F0F9
:1000DE00E8A3F0745A9008A5F0745A9008A6F0D2CE
:1000EE002DC228C22FC22EC22922750B00750A00FE
:1000FE00AE0AAF0BAC08AD09EDC39FEC9E40167473
:10010E00FF12698A75CF01780B740126F650041818
:10011E00E436F650DB22C2AF75D904758F0375B77E
:10012E00A575B7F190F800E4F0758F0175B7A57558
:10013E00B7F1E52790F800F075B7A575B7F190F80F
:10014E0001E4F075B7A575B7F1900899E090F80243
:10015E00F075B7A575B7F190089DE090F803F075AE
:10016E00B7A575B7F190089AE090F804F075B7A5A9
:10017E0075B7F190089BE090F805F075B7A575B7C7
:10018E00F190089CE090F806F075B7A575B7F19060
:10019E00089EE090F807F0758F0075D944D2AF2213
:1001AE00900043E0B4AB61C2AF75D90475B6227549
:1001BE00F522758F0375B7A575B7F1740090F6002B
:1001CE00F0758F01755B00755A00AE5AAF5B7413F4
:1001DE00BE00279F402475B7A575B7F1900885120C
:1001EE000048E0FC90F600120048ECF0785B7401D9
:1001FE0026F6500418E436F650D0758F0075F511BA
:10020E0075B62075D944D2AF22C2AF75F52275D915
:10021E0004755B00755A00AE5AAF5B7413BE0022B4
:10022E009F401F90F600120048E493FC9008851240
:10023E000048ECF0785B740126F6500418E436F6AC
:10024E0050D575D94475F511D2AF22900043E0B464
:10025E00AA028003020396C2AF75D90475B6227541
:10026E00F522758F0375B7A575B7F1740090EE0082
:10027E00F075B7A575B7F1740090F000F075B7A5DD
:10028E0075B7F1740090F200F075B7A575B7F174FB
:10029E000090F400F0758F01755B00755A00AE5A30
:1002AE00AF5B74FFC39F74019E402475B7A575B7ED
:1002BE00F1900073120048E0FC90EE00120048EC42
:1002CE00F0785B740126F6500418E436F650CF75BC
:1002DE005B00755A00AE5AAF5B74FFC39F74019EEC
:1002EE00402475B7A575B7F1900273120048E0FC73
:1002FE0090F000120048ECF0785B740126F6500482
:10030E0018E436F650CF755B00755A00AE5AAF5BE7
:10031E0074FFC39F74019E402475B7A575B7F19005
:10032E000473120048E0FC90F200120048ECF078E2
:10033E005B740126F6500418E436F650CF755B0058
:10034E00755A00AE5AAF5B74FFC39F74019E402472
:10035E0075B7A575B7F1900673120048E0FC90F4DE
:10036E0000120048ECF0785B740126F6500418E495
:10037E0036F650CF758F0075F51175B62075D944C8
:10038E00D2AF743A900773F022900043E0B4AA0201
:10039E0080030204D4C2AF75D90475B62275F52256
:1003AE00758F0375B7A575B7F1740090E600F075FB
:1003BE00B7A575B7F1740090E800F075B7A575B7DD
:1003CE00F1740090EA00F075B7A575B7F17400905E
:1003DE00EC00F0758F01755B00755A00AE5AAF5B7D
:1003EE0074FFC39F74019E402475B7A575B7F19035
:1003FE000073120048E0FC90E600120048ECF07822
:10040E005B740126F6500418E436F650CF755B0087
:10041E00755A00AE5AAF5B74FFC39F74019E4024A1
:10042E0075B7A575B7F1900273120048E0FC90E81D
:10043E0000120048ECF0785B740126F6500418E4C4
:10044E0036F650CF755B00755A00AE5AAF5B74FF2F
:10045E00C39F74019E402475B7A575B7F1900473C0
:10046E00120048E0FC90EA00120048ECF0785B7451
:10047E000126F6500418E436F650CF755B00755A17
:10048E0000AE5AAF5B74FFC39F74019E402475B7D4
:10049E00A575B7F1900673120048E0FC90EC0012BF
:1004AE000048ECF0785B740126F6500418E436F63A
:1004BE0050CF758F0075F51175B62075D944D2AF32
:1004CE00743A900773F022C2AF75D90475F5227590
:1004DE005B00755A00AE5AAF5B74FFC39F74019EEA
:1004EE00401F90EE00120048E493FC90007312003F
:1004FE0048ECF0785B740126F6500418E436F6509A
:10050E00D4755B00755A00AE5AAF5B74FFC39F740F
:10051E00019E401F90F000120048E493FC9002737D
:10052E00120048ECF0785B740126F6500418E4369D
:10053E00F650D4755B00755A00AE5AAF5B74FFC3AC
:10054E009F74019E401F90F200120048E493FC90AD
:10055E000473120048ECF0785B740126F650041810
:10056E00E436F650D4755B00755A00AE5AAF5B7424
:10057E00FFC39F74019E401F90F400120048E49345
:10058E00FC900673120048ECF0785B740126F6506E
:10059E000418E436F650D475F51175D944D2AF74FB
:1005AE003A900773F0C22B22C2AF75D90475F522AB
:1005BE00755B00755A00AE5AAF5B74FFC39F740132
:1005CE009E401F90E600120048E493FC90007312C8
:1005DE000048ECF0785B740126F6500418E436F609
:1005EE0050D4755B00755A00AE5AAF5B74FFC39F53
:1005FE0074019E401F90E800120048E493FC9002A4
:10060E0073120048ECF0785B740126F6500418E47F
:10061E0036F650D4755B00755A00AE5AAF5B74FF58
:10062E00C39F74019E401F90EA00120048E493FCA1
:10063E00900473120048ECF0785B740126F65004B7
:10064E0018E436F650D4755B00755A00AE5AAF5B9F
:10065E0074FFC39F74019E401F90EC00120048E48B
:10066E0093FC900673120048ECF0785B740126F64A
:10067E00500418E436F650D475F51175D944D2AF3E
:10068E00743A900773F0D22B22E54E64046006E5AF
:10069E009964FF60028031A22A4004D22A8027E5A5
:1006AE004E600874E6254E900047F0E54D600874E4
:1006BE00F0254D900047F0E54EB4010280FE754ED8
:1006CE0000754D00C22A8002C22AE54E903280F893
:1006DE00282873754E00E599B4FF03754D01E59911
:1006EE00B4FE03754D02E599B4FD03754D03E5990E
:1006FE00B4FC03754D04E599B4FA03754D05E599FF
:10070E00B4FB06754E01123C4FE599B4F906754ED1
:10071E0004123C4FE599D394E54007E599C394F054
:10072E004002801685994F754E027E017F00E54F7F
:10073E00C394E61269AA8E328F3390087DE4F0A33B
:10074E00F0E599D394C44007E599C394E64002803E
:10075E002885994F754E0374E5C3954FF533753261
:10076E0000AE32AF3390631D126979E493F87401D1
:10077E009390087DC8F0A3C8F0D299020B77900829
:10078E0085E0700AA220B35005A221B34002804238
:10079E0090087DE0FEA3E0FF74FFBE00039F5009AA
:1007AE00EFC39446EE9406401190087DE0FEA3E060
:1007BE00FFEFD3946DEE9406401390087DE0FEA3F8
:1007CE00E0FF900073120048E599F080038599745C
:1007DE00801190087DE0FEA3E0FF900073120048A8
:1007EE00E599F090087D1269B890087DE0FEA3E0CF
:1007FE00FFEFB40106EEB407028003020970900702
:10080E0073E0B43C028003020970A220B35005A22B
:10081E0021B340030208E7C29C900885E0900111C5
:10082E00F0900886E0900080F0900887E09000A09D
:10083E00F0900888E09000C9F0900889E09000756B
:10084E00F090088AE09000BBF090088BE09000D901
:10085E00F090088CE09000ADF090088DE09000CB09
:10086E00F090088EE09000FBF090088FE090015F12
:10087E00F0900890E0900160F0900891E090016196
:10088E00F012358390005EE09000E2F090005FE0A1
:10089E00900099F0900060E090009AF074AB900098
:1008AE0043F01201AE74AA900043F0A22BB34005A0
:1008BE001203978003120259900043E4F090015FF7
:1008CE00E0700C900160E07006900161E0600280C3
:1008DE0004C2208002D220807EC29C900111E09042
:1008EE000885F0900080E0900886F09000A0E090DF
:1008FE000887F09000C9E0900888F0900075E090AD
:10090E000889F09000BBE090088AF09000D9E09042
:10091E00088BF09000ADE090088CF09000CBE0904A
:10092E00088DF09000FBE090088EF0740090088F18
:10093E00F07400900890F07400900891F074AB90F1
:10094E000043F01201AE74AA900043F01202591245
:10095E0003977599FB80FED29C754E00754D007500
:10096E0099FB020B7790087DE0FEA3E0FFEF4E703F
:10097E000685993175300090087DE0FEA3E0FF7486
:10098E00016F4E701BAC30AD31AA32AB33ED2BFB89
:10099E00EC3AFA8A068B07900073120048E599F03C
:1009AE0090087D1269B890087DE0FEA3E0FF740206
:1009BE006F4E7021AC30AD3174566D4C7006E54FF4
:1009CE0064E660028003123C4F123583854F9975A1
:1009DE004E00754D00020B7790087DE0FEA3E0FF00
:1009EE00900073120048E599F090087D1269B89056
:1009FE00087DE0FEA3E0FFAC32AD338F028E038C98
:100A0E00068D07906361126979E493F9740193FE80
:100A1E00EAD39EEB994009854F99754E00754D00AE
:100A2E00020B7790087DE0FEA3E0FF9000731200AA
:100A3E0048E599F090087D1269B890087DE0FEA314
:100A4E00E0FFEFB40006EEB401028003020B7790D4
:100A5E000053E0D394C7400B900053E0C394C8F505
:100A6E0050801A900053E0D39463400B900053E0F3
:100A7E00C39464F5508006900053E0F550E5507530
:100A8E00F002A4FFAEF08F73EF9000731269DBEFEC
:100A9E00FCE0FDEC9000761269DBEDFCE0FDEC2D48
:100AAE00B550028003020B680FEF9000731269DBE2
:100ABE00E573FFE0FCEF9000771269DBECFFE0FCE2
:100ACE00EFC39CB550028003020B68E5739000756E
:100ADE001269DBE573FFE0FCEF9000781269DBEC46
:100AEE00FFE0FCEF2CB55072E5739000791269DBD4
:100AFE00E0C39550900899F0E57390007A1269DB87
:100B0E00E0C3955090089AF0E57390007D1269DB72
:100B1E00E0C3955090089BF0E57390007E1269DB60
:100B2E00E0C3955090089CF0E57390007F1269DB4E
:100B3E00E0C3955090089DF0E5739000801269DB3C
:100B4E00E0C3955090089EF01201247599F97464D3
:100B5E00F5097508001200F880FE7599FF7464F5AA
:090B6E00097508001200F880FE70
:0F3280000206E102078C0209730209E6020A3115
:100B770022E54D90328FF8282873020C5C90087D8F
:100B8700E0FEA3E0FF900049120048E0F5999008C5
:100B97007D1269B890087DE0FEA3E0FF74116F4EE7
:100BA7007003754D00020C5C856E99020C5C900811
:100BB7007DE0FEA3E0FF900073120048E0F599EF97
:100BC700B40107EEB40703754D0090087D1269B8AC
:070BD700020C5C90087EE0B7
:0F328F00020B81020B84020BAF020BB5020BDAAC
:100BDE009032E3F82828738553998067855F998052
:100BEE0062856199805D8565998058856799805386
:100BFE00856899804E8569998049856A9980449067
:100C0E000018E0F599803CA22CB340077599FAC202
:100C1E002C8017A21FB3400575990F800B900047CB
:100C2E00E0F599900047E4F0C21F8017856B99801C
:100C3E0012856699800D856C9980087599FC8003E4
:030C4E00754D00E1
:1032E300020BE5020BEA020BEF020BF4020BF902ED
:1032F3000BFE020C03020C08020C0D020C15020C4F
:0D3303003A020C3F020C44020C49020C4E31
:0B0C510090087D1269B880031233ED9B
:03329E00020C59C6
:100C5C0022E537255BFFAE5A50010E90007312004F
:100C6C0048E0F538E537255BFFAE5A50010E0FBF53
:100C7C0000010E900073120048E0F539853F3BE50A
:100C8C0038B539058538378041E539D39538401D5D
:100C9C00E539C39538853AF0A4FFAEF0E53B8E04F8
:100CAC008F05FF12699AED2538F537801DE538C39D
:100CBC009539853AF0A4FFAEF0E53B8E048F05FF25
:100CCC0012699AEDF4042538F53722E539D39538B5
:100CDC00401DE539C39538853AF0A4FFAEF0E53BED
:100CEC008E048F05FF12699AED2538F537801DE5C6
:100CFC0038C39539853AF0A4FFAEF0E53B8E048FEE
:100D0C0005FF12699AEDF4042538F5372290007925
:100D1C00E0B40170E56775F00A84FF7E008F37E55B
:100D2C006775F00A84ADF07C008D3A753F0A755AF0
:100D3C0005755B24E537C394115005120C5D8006D4
:100D4C009005A8E0F537E537900063F0E56775F09E
:100D5C000A84FF7E008F37E56775F00A84ADF07C5E
:100D6C00008D3A753F0A755A05755B5AE537C39481
:100D7C00115005120C5D80069005DEE0F537E53765
:100D8C0090000EF022900079E0B4016AE56775F0EE
:100D9C000A84FF7E008F37E56775F00A84ADF07C1E
:100DAC00008D3A753F0A755A05755B36E537C39465
:100DBC00115005120C5D80069005BAE0F5378537A9
:100DCC004BE56775F00A84FF7E008F37E56775F099
:100DDC000A84ADF07C008D3A753F0A755A05755B37
:100DEC0048E537C394115005120C5D80069005CC74
:100DFC00E0F53785374C22E55F75F00484FF7E0003
:100E0C008F37E55F75F00484ADF07C008D3A753F4B
:100E1C0004755A01755B00E537C3943F5005120CFD
:100E2C005D80069001B2E0F5378537297528009072
:100E3C000046E075F020A4FFAEF09000C4E08E04F4
:100E4C008F05FF12699A8D379000ACE0D3955F50F7
:100E5C0003020F099000D0E0D3955F4010ED900194
:100E6C00B31269DBE0F52B752A00020F0690009B8C
:100E7C00E0D3955F4043E5379001B31269DBE0F5B1
:100E8C0038E5379001D31269DBE0F5399000D0E0FA
:100E9C00F404255FF53A90009BE0FE9000D0E0F45E
:100EAC00042EF53BE538B539058538378003120C2F
:100EBC00D785372B752A008041E5379001D312690D
:100ECC00DBE0F538E5379001F31269DBE0F539909A
:100EDC00009BE0F404255FF53A9000ACE0FE900036
:100EEC009BE0F4042EF53BE538B5390585383780A1
:100EFC0003120CD785372B752A00020FB09000D344
:100F0C00E0D3955F5011E5379002331269DBE0F5C1
:100F1C002B752A00020FB090009CE0D3955F5043D4
:100F2C00E5379002131269DBE0F538E537900233B0
:100F3C001269DBE0F53990009CE0F404255FF53A8A
:100F4C009000D3E0FE90009CE0F4042EF53BE538D5
:100F5C00B539058538378003120CD785372B752AA0
:100F6C00008041E5379001F31269DBE0F538E53795
:100F7C009002131269DBE0F5399000ACE0F4042523
:100F8C005FF53A90009CE0FE9000ACE0F4042EF586
:100F9C003BE538B539058538378003120CD78537D2
:100FAC002B752A00229000E4E0F53C753F11755A30
:100FBC0002755B00AE52AF53E53C75F00FA4FDAC6F
:100FCC00F0EDD39FEC9E4021E53C8E048F05FF1283
:100FDC00699AED75F010A4FFAEF0E55F75F0118421
:100FEC00FD7C00ED2FF53D800EE55F75F01184FF63
:100FFC007E00EF24F0F53D853D37E55F75F01184FB
:10100C00AFF07E008F3A120C5D85373EAE52AF5377
:10101C009000E4E075F00FA4FDACF0EDD39FEC9ED6
:10102C004028755A02755B10853D37120C5D853E64
:10103C0038853739AE52AF53E53C8E048F05FF121D
:10104C0069C58D3A853C3B120CD78537297528002C
:10105C00752B64752A00229000E4E0F53C753F1175
:10106C00755A02755B00AE52AF53E53C75F00FA498
:10107C00FDACF0EDD39FEC9E4021E53C8E048F053A
:10108C00FF12699AED75F010A4FFAEF0E56175F0F2
:10109C001184FD7C00ED2FF53D800EE56175F0119E
:1010AC0084FF7E00EF24F0F53D853D37E56175F05A
:1010BC001184AFF07E008F3A120C5D85373EAE5234
:1010CC00AF539000E4E075F00FA4FDACF0EDD39FAE
:1010DC00EC9E4028755A02755B10853D37120C5DED
:1010EC00853E38853739AE52AF53E53C8E048F05BB
:1010FC00FF1269C58D3A853C3B120CD78537297593
:10110C002800E56B6017E56BC394FE50109000D877
:10111C00E0B402099000C6E0D3940B50028017AEE5
:10112C0028AF29E56B1269AA74E78E048F05FF12AC
:10113C00699A8C288D299000AEE0B40453E55F7554
:10114C00F00484FF7E008F37E55F75F00484ADF00A
:10115C007C008D3A753F04755A01755B00E537C309
:10116C00943F5005120C5D80069001B2E0F537AE4D
:10117C0028AF29E5371269AA74648E048F05FF1213
:10118C00699AAE28AF29EF2DFDEE3CFC8C288D29F9
:10119C00752B64752A0022900079E0B40146E5674E
:1011AC0075F00A84FF7E008F37E56775F00A84AD11
:1011BC00F07C008D3A753F0A755A05755B00E53772
:1011CC00C394115005120C5D8006900584E0F53730
:1011DC00AE2AAF2BE5372FFF50010E74641269ED68
:1011EC008E2A8F2B90007AE0B40146E56875F00AE0
:1011FC0084FF7E008F37E56875F00A84ADF07C00C3
:10120C008D3A753F0A755A05755B6CE537C39411B9
:10121C005005120C5D80069005F0E0F537AE2AAF54
:10122C002BE5372FFF50010E74641269ED8E2A8F57
:10123C002B900089E0B40249E56AC3944175F0052E
:10124C0084FF7E008F37E56A75F00584ADF07C0075
:10125C008D3A753F05755A06755B00E537C39413D7
:10126C005005120C5D8006900686E0F537AE2AAF6D
:10127C002BE5372FFF50010E74641269ED8E2A8F07
:10128C002B9000CBE0B402028003021342E55F75A1
:10129C00F01584FF7E008F37E55F75F01584ADF097
:1012AC007C008D3A753F15755A03755BF4E537C3B1
:1012BC00940B5005120C5D8006900472E0F537E536
:1012CC003775F0FFA4FFAEF09000CCE08E048F05D4
:1012DC00FF12699AED90005CF0E56675F078A4FF5A
:1012EC00AEF074FF8E048F05FF12699A8C5A8D5BD9
:1012FC0074028C068D071200398F37AC5AAD5B74B3
:10130C0004FF1269C58D3A753F04755A06755B2842
:10131C00E537C3941D5005120C5D80069006B8E0AD
:10132C00F537AE2AAF2BE5372FFF50010E74641240
:10133C0069ED8E2A8F2B900078E0B4025DE5617523
:10134C00F064A4FFAEF074081200398E5C8F5D74EB
:10135C00058E048F05FF12699A8D37AE5CAF5D74F4
:10136C00058E048F05FF1269C58D3A753F05755AB8
:10137C0005755BDEE537C394135005120C5D8006D2
:10138C00900664E0F537AE2AAF2BE5372FFF5001FE
:10139C000E74641269ED8E2A8F2B9000BAE0703CAB
:1013AC00900046E075F00584FF7E008F3790004674
:1013BC00E075F00584ADF07C008D3A753F05755AEB
:1013CC0005755BC0E537C3941D5005120C5D800696
:1013DC00900650E0F537E537900064F022900081DC
:1013EC00E0B401179008A0E0252BFFAE2A50010EA7
:1013FC009000D5E01269ED8E2A8F2B9000F9E0B4A5
:10140C0001149000FAE0A852B8000495535007E577
:10141C005FC39560400280139000A3E0252BFFAEC4
:10142C002A50010E8E2A8F2B021818900081E0B4DE
:10143C000306A228B3B3400280509008A9E07010B4
:10144C009008A3E0C39405A852B800069553400237
:10145C0080109000A3E0252BFFAE2A50010E8E2A9F
:10146C008F2B9008A9E0600D9008A3E0A852B8005B
:10147C00069553400280109000A3E0252BFFAE2A66
:10148C0050010E8E2A8F2B02181890007BE0B402AC
:10149C0002800302181890007EE0602FE567D39459
:1014AC0046402890000FE0FEA3E0FF9000B9E075E5
:1014BC00F003A4FDACF0EFD39DEE9C400E9000DD4C
:1014CC00E0A852B80005D3955350030218189000A9
:1014DC00AEE0B40302800302167C85615B755A0092
:1014EC00900085E0A852B800049553500E900086E9
:1014FC00E0A85AB80005D3955B5003021679E56154
:10150C0075F002A4FFAEF074158E048F05FF1269FE
:10151C009A8C068D07900603120048FEE0FFEE90B1
:10152C00007DE0FEEF8E0088F0A4FFAEF074648EB8
:10153C00048F05FF12699A8C5A8D5B900046E075FA
:10154C00F018A4FFAEF09000C4E08E048F05FF12DB
:10155C00699A8C068D0790061B120048AE5AAF5B39
:10156C00E01269AA74648E048F05FF12699A8C5A72
:10157C008D5BE565A85AB80077D3955B4072E5653D
:10158C00C3955BFFE4955AFE8E5A8F5B7428BE00A0
:10159C00039F500C755B28755A00740D900047F032
:1015AC00AE5AAF5B90007EE01269AA74288E048F4D
:1015BC0005FF12699A8C5A8D5BAE28AF29740A8E7E
:1015CC00048F05FF12699A8D068C07AC5AAD5BCF60
:1015DC00CECF120003740A8E048F05FF12699A8C09
:1015EC005A8D5BAE28AF291269F58E288F29807D24
:1015FC00E565A85AB80004955B5072AE5AAF5BE52E
:10160C00651269ED8E5A8F5B7428BE00039F500CD7
:10161C00755B28755A00740D900047F0AE5AAF5B9D
:10162C0090007EE01269AA74288E048F05FF12695F
:10163C009A8C5A8D5BAE28AF29740A8E048F05FFE5
:10164C0012699A8D068C07AC5AAD5BCFCECF1200C7
:10165C0003740A8E048F05FF12699A8C5A8D5BAE47
:10166C0028AF29EF2DFDEE3CFC8C288D2902181893
:10167C009000C6E0855FF0A4FFAEF074051269AA75
:10168C0074071200398E5A8F5B900085E0A852B80F
:10169C00000495535012900086E075F002A4FDAC46
:1016AC00F0EFC39DEE9C4003021818E55F75F00B3C
:1016BC0084FF7E00900603120048FEE0FFEE9000CF
:1016CC007DE0FEEF8E0088F0A4FFAEF074648E0413
:1016DC008F05FF12699A8C5A8D5B900046E075F06D
:1016EC0018A4FFAEF09000C4E08E048F05FF1269C1
:1016FC009A8C068D0790061B120048AE5AAF5BE021
:10170C001269AA74648E048F05FF12699A8C5A8D23
:10171C005BE565A85AB80077D3955B4072E565C365
:10172C00955BFFE4955AFE8E5A8F5B7428BE0003BE
:10173C009F500C755B28755A00740D900047F0AEE5
:10174C005AAF5B90007EE01269AA74288E048F0554
:10175C00FF12699A8C5A8D5BAE28AF29740A8E04DD
:10176C008F05FF12699A8D068C07AC5AAD5BCFCEF4
:10177C00CF120003740A8E048F05FF12699A8C5ADB
:10178C008D5BAE28AF291269F58E288F29807DE5F7
:10179C0065A85AB80004955B5072AE5AAF5BE5650C
:1017AC001269ED8E5A8F5B7428BE00039F500C7526
:1017BC005B28755A00740D900047F0AE5AAF5B90E1
:1017CC00007EE01269AA74288E048F05FF12699AB4
:1017DC008C5A8D5BAE28AF29740A8E048F05FF12CC
:1017EC00699A8D068C07AC5AAD5BCFCECF12000335
:1017FC00740A8E048F05FF12699A8C5A8D5BAE2881
:10180C00AF29EF2DFDEE3CFC8C288D29229000D9C0
:10181C00E0B4026AE55F75F00884FF7E008F37E55F
:10182C005F75F00884ADF07C008D3A753F08755AF1
:10183C0001755BE0E537C3943F5005120C5D8006E3
:10184C00900272E0F53785372D752C00AE2CAF2D3C
:10185C00AC2AAD2B12000374648E048F05FF126941
:10186C009A8C2C8D2D900076E08C068D071269AA2F
:10187C0074648E048F05FF12699A8C2C8D2DAE2802
:10188C00AF29AC2AAD2B12000374648E048F05FFB4
:10189C0012699A8C288D29900076E08C068D07129F
:1018AC0069AA74648E048F05FF12699A8C288D299D
:1018BC00A204401DAE52AF537405BE00039F5002EC
:1018CC00D204E561D394CC4008D202741190004745
:1018DC00F09000D8E0B402089000C6E0640B6002FF
:1018EC008035AE28AF29E56B1269AA74E78E048F98
:1018FC0005FF12699A8C288D299000D9E0B4021743
:10190C00AE2CAF2DE56B1269AA74E78E048F05FF20
:10191C0012699A8C2C8D2D900098E05402601B90CB
:10192C00008FE0A852B80012D39553400DA204B317
:10193C00B35007E561C3949A40028028AE34AF35AA
:10194C0090008DE075F002A4FDACF0EF2DFDEE3CA7
:10195C00FC74022DFD50010CE561BC0007D39D40C9
:10196C0003754301856135753400E5437003021A34
:10197C005C9000EBE0C395435003021A4E9000FBC1
:10198C00E0C394025076E56775F00A84FF7E009000
:10199C000573120048E0F55B755A00AE5AAF5B90C8
:1019AC00008EE01269AA74648E048F05FF12699A86
:1019BC008C5C8D5D9000EBE004C395438C068D0729
:1019CC001269AA9000EBE08E048F05FF12699A8CC5
:1019DC005C8D5DAE28AF29EF2DFDEE3CFC8C288D87
:1019EC00299000D9E0B40212AE2CAF2DAA5CAB5DED
:1019FC00EF2BFBEE3AFA8A2C8B2D80469000EBE015
:101A0C0004C39543854BF0A4FFAEF09000EBE08E41
:101A1C00048F05FF12699A8C5C8D5DAE28AF29EF9F
:101A2C002DFDEE3CFC8C288D299000D9E0B40212DF
:101A3C00AE2CAF2DAA5CAB5DEF2BFBEE3AFA8A2CE9
:101A4C008B2D05439000EBE0C39543500375430089
:101A5C00900098E05401601B90008CE0A852B800F4
:101A6C0012D39553400DA204B3B35007E55FC39452
:101A7C00CC4002802590008AE075F003A4FFAEF004
:101A8C00E5402FFF50010E74032FFF50010EE55F50
:101A9C00BE0007D39F4003754401855F40E5447049
:101AAC0003021B8F9000ECE0C395445003021B8192
:101ABC009000FBE0C394025076E56775F00A84FF52
:101ACC007E00900573120048E0F55B755A00AE5A23
:101ADC00AF5B90008BE01269AA74648E048F05FFD3
:101AEC0012699A8C5C8D5D9000ECE004C395448C7B
:101AFC00068D071269AA9000ECE08E048F05FF1288
:101B0C00699A8C5C8D5DAE28AF29EF2DFDEE3CFC07
:101B1C008C288D299000D9E0B40212AE2CAF2DAADE
:101B2C005CAB5DEF2BFBEE3AFA8A2C8B2D8046904A
:101B3C0000ECE004C39544854CF0A4FFAEF090009B
:101B4C00ECE08E048F05FF12699A8C5C8D5DAE28DB
:101B5C00AF29EF2DFDEE3CFC8C288D299000D9E0AF
:101B6C00B40212AE2CAF2DAA5CAB5DEF2BFBEE3AA0
:101B7C00FA8A2C8B2D05449000ECE0C3954450035D
:101B8C007544009000EEE02529FFAE2850010E8E22
:101B9C00288F2990009DE0A828B8000495295009A9
:101BAC0090009DE0F5297528009000D9E0B4020D55
:101BBC0090009DE0A82CB80006952D40028009905D
:101BCC00009DE0F52D752C00229000D9E0B40102A7
:101BDC008003021CE0A204B35003021CDE9000A49C
:101BEC00E0B40168AE28AF29AC52AD5312000374B7
:101BFC003C8E048F05FF12699A9000B4E0BC001073
:101C0C009D400D9000B6E0A828B80004952950021C
:101C1C00D203AE28AF29AC52AD53120003743C8EE4
:101C2C00048F05FF12699A9000B4E0C3940ABC00BB
:101C3C0015D39D40119000B6E0C39405A828B800B8
:101C4C0005D3952950028002C2038068AE28AF29C3
:101C5C00AC52AD5312000374788E048F05FF1269D9
:101C6C009A9000B4E0BC00109D400D9000B6E0A826
:101C7C0028B8000495295004D2038038AE28AF2927
:101C8C00AC52AD5312000374788E048F05FF1269A9
:101C9C009A9000B4E0C3940ABC0015D39D401190F7
:101CAC0000B6E0C39405A828B80005D395295002C6
:101CBC008002C203A203B34019AE28AF299000B52D
:101CCC00E01269AA74648E048F05FF12699A8C283D
:101CDC008D298002C203A201B34006A202B3B35005
:101CEC0009900017E4F0A3F08024AE28AF2974000B
:101CFC00D39F74019E400C900017E528F0A3E529B2
:101D0C00F0800B74FF900017F8E4F0E8A3F090005B
:101D1C00A4E0B4011AAE28AF2974021269AA8E2865
:101D2C008F29AE2CAF2D74021269AA8E2C8F2D9098
:101D3C0000BBE0C39403400990006FE0C3940250D1
:101D4C0035AE28AF29745E1269AA740A8E048F0509
:101D5C00FF12699A8C288D299000D9E0B40217AE35
:101D6C002CAF2D745E1269AA740A8E048F05FF12B3
:101D7C00699A8C2C8D2DAE28AF297402BE000AD323
:101D8C009F4006752902752800AE2CAF2D7402BE3B
:101D9C00000AD39F4006752D02752C00900015E5A6
:101DAC0028F0A3E529F022900046E0900373126915
:101DBC00DBE0F541754264900046E0FE9000AFE038
:101DCC00D39E4037E55F75F00884FF7E008F37E5C2
:101DDC005F75F00884ADF07C008D3A753F08755A3C
:101DEC0003755B96E537C3941F5005120C5D800696
:101DFC00900428E0F5378537428035E55F75F008AB
:101E0C0084FF7E008F37E55F75F00884ADF07C00B1
:101E1C008D3A753F08755A03755BB6E537C3941F49
:101E2C005005120C5D8006900448E0F5378537426A
:101E3C00229000E5E0F53C753F11755A04755B0086
:101E4C00AE52AF53E53C75F00FA4FDACF0EDD39F53
:101E5C00EC9E4021E53C8E048F05FF12699AED75CE
:101E6C00F010A4FFAEF0E55F75F01184FD7C00ED81
:101E7C002FF53D800EE55F75F01184FF7E00EF2499
:101E8C00F0F53D853D37E55F75F01184AFF07E00D0
:101E9C008F3A120C5D85373EAE52AF539000E5E0A1
:101EAC0075F00FA4FDACF0EDD39FEC9E4028755A55
:101EBC0004755B10853D37120C5D853E38853739CE
:101ECC00AE52AF53E53C8E048F05FF1269C58D3AB7
:101EDC00853C3B120CD7853741754264229000E556
:101EEC00E0F53C753F11755A04755B00AE52AF536B
:101EFC00E53C75F00FA4FDACF0EDD39FEC9E4021BA
:101F0C00E53C8E048F05FF12699AED75F010A4FF65
:101F1C00AEF0E56175F01184FD7C00ED2FF53D8090
:101F2C000EE56175F01184FF7E00EF24F0F53D8520
:101F3C003D37E56175F01184AFF07E008F3A120CDD
:101F4C005D85373EAE52AF539000E5E075F00FA4BF
:101F5C00FDACF0EDD39FEC9E4028755A04755B10D8
:101F6C00853D37120C5D853E38853739AE52AF53FF
:101F7C00E53C8E048F05FF1269C58D3A853C3B12FA
:101F8C000CD78537417542649000E0E0B404799039
:101F9C000046E0FE9000AFE0D39E4037E55F75F061
:101FAC000884FF7E008F37E55F75F00884ADF07C08
:101FBC00008D3A753F08755A03755B96E537C394E7
:101FCC001F5005120C5D8006900428E0F53785370C
:101FDC00428035E55F75F00884FF7E008F37E55F42
:101FEC0075F00884ADF07C008D3A753F08755A0386
:101FFC00755BB6E537C3941F5005120C5D800690D7
:10200C000448E0F53785374222900079E0B4013B73
:10201C00E56775F00A84FF7E008F37E56775F00A77
:10202C0084ADF07C008D3A753F0A755A05755B12CC
:10203C00E537C394115005120C5D8006900596E0AF
:10204C00F537E5422537C39464F54290007AE0B445
:10205C00013BE56875F00A84FF7E008F37E56875F3
:10206C00F00A84ADF07C008D3A753F0A755A0575FF
:10207C005B7EE537C394115005120C5D800690060B
:10208C0002E0F537E5422537C39464F542E5412576
:10209C0042F536900081E0B4021090089FE025369E
:1020AC00FE9000D5E0F4042EF5369000D8E0D394E1
:1020BC00014040E56BC394E7501D74E7C3956BFE7C
:1020CC009008A1E08E00F5F0E884FF7E008F37E5E4
:1020DC00362537F536801CE56BC394E7FE9008A1D6
:1020EC00E08E00F5F0E884FF7E008F37E536C3956F
:1020FC0037F536A2044006E5412464F536E536D3BF
:10210C0094644009E536C39464F536800375360053
:10211C009000B1E0C3953650069000B1E0F5362240
:10212C00D201900062E0A852B800049553503E9042
:10213C000062E0A852B800049553500375360F9016
:10214C000062E004A852B80004955350037536079A
:10215C00900062E02402A852B8000495535002C2C9
:10216C0001900062E060067409900047F0C22F7E77
:10217C00017F009000B7E01269AA9000C6E08E04BF
:10218C008F05FF12699AE55FBC0017D39D40139031
:10219C0000C0E0B40204D22F8002C201740A900085
:1021AC0047F0900079E0B401099000B8E0C395675E
:1021BC00400280159000CAE0A852B8000495535014
:1021CC0002C201740B900047F0900079E0B4010753
:1021DC00E567C394644002801D900110E0600D908F
:1021EC000110E0A852B80006955340028008C201C5
:1021FC00740B900047F0A20140037536009000F973
:10220C00E0B401149000FAE0A852B80004955350C1
:10221C0007E55FC39560400280209000A2E0D39454
:10222C001D400B9000A2E0C3941EF536800375365A
:10223C00007415900047F002231D900081E0B40358
:10224C0006A228B3B3400302231D9008A3E0C39455
:10225C0005A852B80004955350069008A9E06002F6
:10226C00801D9000A2E0D3941D400B9000A2E0C30F
:10227C00941EF5368003753600740C900047F09070
:10228C0008A3E0A852B80004955350069008A9E0A2
:10229C007002801D9000A2E0D3941D400B9000A210
:1022AC00E0C3941EF5368003753600740C9000471D
:1022BC00F09008A3E0A852B8000495535031900058
:1022CC00C0E0B40228D22F9008A8E0FE9008A9E044
:1022DC00D39E50069008A9E0700280099008A8E4EB
:1022EC00F0C22F80069008A8E004F08002C2019092
:1022FC0008A3E02405A852B800049553501390008D
:10230C00C0E0B4020A9008A9E07002D22F8002C289
:10231C0001A22EB3401D9000A2E0D3941D400B905F
:10232C0000A2E0C3941EF53680037536007410903D
:10233C000047F085366C9000A2E0D3941D401890B5
:10234C000070E02536FE900046E075F01E84FC7FA0
:10235C0000EE2CF5368049900047E0640C600F903D
:10236C000047E064106007900047E0B41516900039
:10237C0070E0FE900046E075F01E84FC7F00EE2CB1
:10238C00F536801C900072E02536FE900070E02E31
:10239C00FE900046E075F01E84FC7F00EE2CF536B6
:1023AC0022900046E075F00584FF7E008F37900088
:1023BC0046E075F00584ADF07C008D3A753F0575EF
:1023CC005A03755BD69000C4E01475F00584FF7E4B
:1023DC0000E537BE00039F5005120C5D800BE537FE
:1023EC009004491269DBE0F537E5379008A2F090CC
:1023FC0008A2E0FE9000B3E0C39E50089000B3E04A
:10240C009008A2F022E56775F00A84FF7E00900523
:10241C0073120048E0F546E546D394644010E54657
:10242C00C3946475F00F84FF7E008F46800375465D
:10243C0000900096E02546F54622E56775F00A8483
:10244C00FF7E00900573120048E0C39469505590CC
:10245C0000E0E0C394035026900875E0FEA3E0FF73
:10246C007404120039E55F1269AA740F8E048F058B
:10247C00FF12699A900873ECF0A3EDF08024900899
:10248C0075E0FEA3E0FF7404120039E5611269AA3D
:10249C00740F8E048F05FF12699A900873ECF0A3E9
:1024AC00EDF0800F900875E0F8A3E0900873C8F089
:1024BC00A3C8F0A204401A900875E0FEA3E0FF74D4
:1024CC00031269AA7401120039900873EEF0A3EF9D
:1024DC00F0900873E0FEA3E0FF900879E0FCA3E025
:1024EC00FDEDD39FEC9E400F900879E0F8A3E090AF
:1024FC000873C8F0A3C8F0900089E0B40262E56AE2
:10250C00C3944175F00584FF7E008F37E56A75F042
:10251C000584ADF07C008D3A753F05755A06755BE8
:10252C0014E537C394175005120C5D800690069A7B
:10253C00E0F537900873E0FEA3E0FF740A8E048F79
:10254C0005FF12699AE5378C068D071269AA740A81
:10255C008E048F05FF12699A900873ECF0A3EDF0CE
:10256C0022E50875F004A4FFAEF09006B612004800
:10257C00E09032A1F8282873804C855373804790E3
:10258C0000C6E0855FF0A4FFAEF074081200398F2E
:10259C00738033856173802E85677380298568739A
:1025AC008024856973801F856A73801A856B73809C
:1025BC00158566738010856573800B856C7380063A
:0625CC00900018E0F57319
:1032A10002258402258602258B02259F0225A40280
:1032B10025A90225AE0225B30225B80225BD0225A6
:0732C100C20225C70225CC63
:1025D200E50875F004A4FFAEF09006B7120048E5D6
:1025E2000875F004A4FFAEF0E0FC9006B8120048B3
:1025F200ECFEE0FFEEC39F40030226DAE50875F029
:1026020004A4FFAEF09006B6120048E0B40441E51F
:102612000875F004A4FFAEF09006B8120048E0C3BB
:102622009573500AE508F50CD3923012404FE50835
:1026320075F004A4FFAEF09006B7120048E0D395FF
:1026420073400AE508F50CC3923012404F0226D8B7
:10265200E50875F004A4FFAEF09006B7120048E05A
:10266200C395735015E50875F004A4FFAEF090060B
:10267200B8120048E0D395735002800AE508F50CC1
:10268200D3923012404FE50875F004A4FFAEF090EB
:1026920006B7120048E0D395735015E50875F004AB
:1026A200A4FFAEF09006B8120048E0C39573500A3A
:1026B200E508F50CC3923012404F9006BEE0B4011B
:1026C200099000D2E0D395615002800A7402F50CA1
:1026D200C3923012404F806AE50875F004A4FFAE41
:1026E200F09006B7120048E0D395734015E50875DF
:1026F200F004A4FFAEF09006B8120048E0C3957350
:102702004002800AE508F50CC3923012404FE508FA
:1027120075F004A4FFAEF09006B7120048E0C3952E
:10272200734015E50875F004A4FFAEF09006B812E8
:102732000048E0D39573400AE508F50CD3923012B5
:10274200404F22AE2EAF2F74C9BE000CD39F40085B
:10275200782E1269FD02285F752F01752E00AE5288
:10276200AF53E546BE000DD39F40099000A8E0D3C9
:10277200954740028023754700E546C39553F5739C
:102782009000ABE0D395454008E5452573F54580BB
:10279200069000ABE0F54580020547900084E0D347
:1027A2009561401CE55FC395604015AE52AF53E59D
:1027B20046BE00039F50099000A9E0D3954840020D
:1027C200806E9008A4E0A852B80004955350037597
:1027D2004A009008A4E0A852B8000BD395534006D3
:1027E200E5539008A4F0E54A7041E553C39546F5D8
:1027F20073E573D3940540037573059000AAE0C393
:1028020095455007E573C3954540028009E545C3E8
:102812009573F54580069000AAE0F5459000AAE080
:10282200D3954540069000AAE0F545754800800220
:102832000548E54A7016900084E0C39561500DE5A5
:10284200462405A852B8000695534002800F900016
:1028520097E0F545754A0174789008A4F022AE2EEF
:10286200AF2F74E9D39F74039E4008782E1269FD3E
:10287200022A06752F01752E00754532A229402ABB
:10288200754519900097E075F002A4FFAEF0E54798
:10289200BE0006D39F4002D2290547754A037478C9
:1028A2009008A4F07549000229EDAE52AF53E546F7
:1028B2006F4E70030229EDE546BE000DD39F40091D
:1028C2009000A8E0D395474002800F754700E54A83
:1028D200C394035003754519800DE546C39553F51E
:1028E20073E5472573F547900084E0D39561400E68
:1028F2009008A4E0A852B80007D395534002800C78
:102902000549900097E0B54903754A00E54AB403CA
:1029120006A204B3B34002800A0549E549B43C0368
:10292200754A02E54AB402299008A4E0A852B80008
:102932000ED395534009E5539008A4F075490090D1
:102942000084E0C39561500975490074789008A429
:10295200F0E54A705A900084E0D39561401CE55F2F
:10296200C395604015AE52AF53E546BE00039F507B
:10297200099000A9E0D39548400280087548007587
:10298200454B8028E553C39546F573E573D394050B
:102992004003757305900084E0D395614008E548D3
:1029A2002573F5488006E5482406F548754900E593
:1029B2004A7016900084E0C39561500DE5462405E7
:1029C200A852B80006955340028003754A01E54AB1
:1029D200B401187545190549900097E0B549067587
:1029E2004A0275490074789008A4F0A202B3400329
:1029F200754532E54575F00AA4FFAEF090087BEE0E
:102A0200F0A3EFF022E56F9032C8F8282873900007
:102A12007CE07003022C449000B2E0B40102800317
:102A2200022B4F900044E0655E6009E55345526019
:102A320003022B4C7E017F00E5BE1269AAE5BD2F81
:102A4200FF50010E8E5A8F5B74101269AA900061BA
:102A5200E08E048F05FF12699A90087FECF0A3EDD7
:102A6200F0E56B600FE56BC394FE50089000D8E070
:102A72006402600280649000C6E0B40B1F90087F7D
:102A8200E0FEA3E0FF74E71269AAE56B8E048F05EE
:102A9200FF12699A90087FECF0A3EDF09000C6E077
:102AA200D3940B40089000AEE064046002802B9047
:102AB200087FE0FEA3E0FF900883E0FCA3E0FDEFC7
:102AC200D39DEE9C400D1269F590087FEEF0A3EFC6
:102AD200F0800790087FE4F0A3F090007CE0B4025D
:102AE20027900881E0FEA3E0FF90087FE0FCA3E0CE
:102AF200FDEF2DFDEE3CFC74018C068D07120039B2
:102B020090087FEEF0A3EFF090087FE0FEA3E0FFD5
:102B1200900881E0FCA3E0FDEDD39FEC9E4004D23F
:102B22002D8002B22D90087FE0F8A3E0900881C8C2
:102B3200F0A3C8F09000AEE064016006A22DB3B32A
:102B420040028006900880E0F55F022C42D22D7E82
:102B5200017F00E5BE1269AAE5BD2FFF50010E8E6E
:102B62005A8F5B74101269AA900061E08E048F057F
:102B7200FF12699A90087FECF0A3EDF0E56B600F0D
:102B8200E56BC394FE50089000D8E06402600280B6
:102B9200649000C6E0B40B1F90087FE0FEA3E0FF44
:102BA20074E71269AAE56B8E048F05FF12699A9089
:102BB200087FECF0A3EDF09000C6E0D3940B400840
:102BC2009000AEE064046002802B90087FE0FEA3D8
:102BD200E0FF900883E0FCA3E0FDEFD39DEE9C4074
:102BE2000D1269F590087FEEF0A3EFF080079008D0
:102BF2007FE4F0A3F090007CE0B40227900881E02B
:102C0200FEA3E0FF90087FE0FCA3E0FDEF2DFDEEC8
:102C12003CFC74018C068D0712003990087FEEF09F
:102C2200A3EFF090087FE0F8A3E0900881C8F0A33A
:102C3200C8F09000AEE064016006900880E0F55FA5
:102C42008003755F00900078E07006756F01022ABC
:102C52000775BB1802327B900078E07003022DCA20
:102C62007E017F00E5BE1269AAE5BD2FFF50010E6D
:102C72008E5A8F5B9000BEE0B4010F7E0F7FFFACD7
:102C82005AAD5B1269F58E5A8F5B9000E3E0B40295
:102C920045AE5AAF5B900021E0FCA3E0FDEDD39F6F
:102CA200EC9E400A900021E55AF0A3E55BF0AE5A93
:102CB200AF5B900023E0FCA3E0FDEFD39DEE9C40D0
:102CC2000A900023E55AF0A3E55BF0AE5AAF5B74BD
:102CD200041200398F619000E3E0704CAE5AAF5B92
:102CE200900021E0FCA3E0FDEFD39DEE9C40091291
:102CF20069F58E5A8F5B8006755B00755A00AE5A75
:102D0200AF5B74101269AA90005EE08E048F05FF1B
:102D120012699A8C5A8D5B74FFBC0009D39D4005E1
:102D2200855B6180037561FE9000AEE0B4010280B4
:102D320003022DC8A204B3B3500E900082E0A85241
:102D4200B80005D39553500280719000BFE08561B1
:102D5200F0A4FFAEF074648E048F05FF12699A8CA2
:102D62005A8D5BE56B6016E56BC394FE500F9000C5
:102D7200D8E0B402089000C6E0640B60028017AE8F
:102D82005AAF5B74E71269AAE56B8E048F05FF12D6
:102D9200699A8C5A8D5BAE5AAF5B90087FE0FCA3B8
:102DA200E0FDEDD39FEC9E4005855B5F800BA22D7D
:102DB200B34006900880E0F55F800BA22DB3400679
:102DC200900880E0F55F800375610090007BE07001
:102DD20006756F02022A0775BB1902327B90007BCF
:102DE200E07003022E7FE55ED395514003022E7DF3
:102DF20090001FE0FEA3E0FFE5651269ED90001F61
:102E0200EEF0A3EFF07E017F00E5BE1269AAE5BDF8
:102E12002FFF50010E8E5A8F5B9000E8E070137402
:102E22000A1269AA74518E048F05FF12699A8D6580
:102E32008019AE5AAF5B740A1269AA8F048E057E9E
:102E4200017F95CDCCCD1268988F65E565D39464EA
:102E5200400375656490001FE0FEA3E0FFE5652F67
:102E6200FF50010E90001FEEF0A3EFF090007FE004
:102E7200048E048F05FF12699A8D65800375653291
:102E82009000CBE07006756F03022A0775BB130230
:102E9200327B9000CBE0604A7E017F00E5BE126982
:102EA200AAE5BD2FFF50010E8E5A8F5B74041200EB
:102EB200398F669000CDE08566F0A4FDACF07464B5
:102EC200FF12699A8D669000CCE08566F0A4FFAE91
:102ED200F074FF8E048F05FF12699AED90005DF089
:102EE2008003756600900079E07006756F04022A0F
:102EF2000775BB1702327B900079E0B401028003B0
:102F0200022F8D7E017F00E5BE1269AAE5BD2FFF6B
:102F120050010E8E5A8F5B9008A5E060199008A5AB
:102F2200E0149063A512008CE493FC740193FDED10
:102F3200C39FEC9E400280069008A5E014F0900822
:102F4200A5E0C394B3501DAE5AAF5B9008A5E00450
:102F52009063A512008CE493FC740193FDEFC39D72
:102F6200EE9C400280069008A5E004F09008A5E0DF
:102F7200FE90009FE08E0088F0A4FFAEF074648E95
:102F8200048F05FF12699A8D6780037567009000B0
:102F92007AE07006756F05022A0775BB1602327B4E
:102FA20090007AE0B4010280030230367E017F0095
:102FB200E5BE1269AAE5BD2FFF50010E8E5A8F5B46
:102FC2009008A6E060199008A6E01490650F120020
:102FD2008CE493FC740193FDEDC39FEC9E40028050
:102FE200069008A6E014F09008A6E0C394B3501D22
:102FF200AE5AAF5B9008A6E00490650F12008CE415
:1030020093FC740193FDEFC39DEE9C4002800690F9
:1030120008A6E004F09008A6E0FE9000A5E08E006D
:1030220088F0A4FFAEF074648E048F05FF12699AD3
:103032008D68800375680075BB1F02327B7E017F3D
:1030420000E5BE1269AAE5BD2FFF50010E8E5A8F10
:103052005B74091269AA74E68E048F05FF12699ADD
:103062008D6A900081E07006756F07022A0775BBB2
:103072001502327B900081E070030231C77E017F2E
:1030820000E5BE1269AAE5BD2FFF50010E8E5A8FD0
:103092005B74041200398F69900081E0B4011590CD
:1030A20000D5E08569F0A4FFAEF07407120039EF95
:1030B2009008A0F0900081E0B402159000D5E08560
:1030C20069F0A4FFAEF07407120039EF90089FF088
:1030D200900081E0B4030280030231AA9000C2E0B2
:1030E2007052E569C39419500FD2289000A1E09064
:1030F20008A3F09008A7E4F0E569D394644004A221
:10310200284002802D9008A7E004F09008A7E0FE76
:10311200900114E0B5060B9008A3E004F09008A714
:10312200E4F09008A3E064966006900114E0700257
:10313200C22880639000A1E070349000D5E08569D8
:10314200F0A4FFAEF074FF8E048F05FF12699AEDB2
:103152009008A3F0AE52AF53741EBE0006D39F4038
:1031620002D228E561D394E54002C2288029E569AC
:10317200C3940A500DAE52AF53741EBE0004D39FC7
:1031820050028002D228E561D394E54002C2289021
:1031920000A1E09008A3F09008A3E0C394055006B4
:1031A20074059008A3F0C22E900081E0B40414E5E7
:1031B20069C394195002D22EE569D394324002C2F7
:1031C2002EC22880037569009000D8E07006756FE2
:1031D20008022A0775BB1402327B9000D8E0700304
:1031E20002326A7E017F00E5BE1269AAE5BD2FFFA9
:1031F20050010E8E5A8F5B9000FDE07025EFD39444
:1032020021EE940E4005756BFF8015AE5AAF5B74CC
:10321200101269AA74E38E048F05FF12699A8D6BEE
:103222008027AE5AAF5BEFD39449EE940640057502
:103232006BFF8015AE5AAF5B74101269AA74658E6B
:10324200048F05FF12699A8D6BE56B75F00BA4FF75
:10325200AEF09000C6E08E048F05FF12699A9008C6
:1032620083ECF0A3EDF08003756B0090007CE060CE
:093272000575BB1A800375BB1839
:1032C800022A10022C59022DDF022E94022EF90236
:0B32D8002FA202303F0230760231DCF2
:05327B00056FD2EC22FA
:0969DB002582F582500205832299
:0F008C0025E050020583258250020583F582226C
:10697900EF2F500205832582F582E5833E2EF583AC
:0169890022EB
:1069ED00CFC39FFF50011E22C3EF9DFFEE9CFE22E1
:0869FD000806B600021806228C
:0D69B800A3E004F070061269D1E004F022A3
:0E003900048007C3CE13CECF13CFD5E0F6223E
:10689800BC000FBE0008ED8FF084FFADF022E4FECF
:1068A800FF22BE000DEF60FE54F0606F20E7030288
:1068B800694EEAC0E0EBC0E078017A0075F001EEBD
:1068C80020E710EF25E0FFEE33FE0AC5F023C5F000
:1068D80030E7F0EA5407F9096A7A007B006001089A
:1068E800C3EC9E40167004ED9F4010ED9FFDEC9E9A
:1068F800FCE5F0CA4ACA03F5F08005E5F003F5F0B7
:10690800C3EE13FEEF13FFD9D77908CACBCAD8D084
:10691800EAFEEBFFD0E0FBD0E0FA22EC8FF084FC3B
:10692800ED54F045F0C48FF084FEEDC454F045F00A
:10693800C48FF084FDEEC4FE54F02DFFEE540F3CDE
:10694800FEADF07C0022790078008FF0EC7E082004
:10695800E70DC3CD33CD33C933C9C833C8DEF0849E
:1069680049F9E5F08FF0BE00E6FD7C00E9FFE8FE9E
:0169780022FC
:0E69AA00F88FF0A4FFE5F0CE88F0A42EFE22B8
:10000300EF8DF0A4F9A8F0EF8CF0A428F8EE8DF0B2
:06001300A428FEE9FF2213
:10698A00600D782B026994007830D8FED5E0F822A1
:10699A00EEC0E07E00126898EFFDEEFCD0E0FE2229
:0C69C500EEC0E07E00126898D0E0FE22D8
:03001B0002001EC2
:0300530002005652
:03009B00020071EF
:030000000269E4AE
:0969E40075817575D0000242EBCB
:0B004800E5822FF582E5833EF5832260
:0A69D1000582D5820215831582228B
:10001E00C0E0C0F0C083C082C0D075D0001241E9EC
:0B002E00D0D0D082D083D0F0D0E032E0
:10005600C0E0C0F0C083C082C0D075D0001241ECB1
:10006600D0D0D082D083D0F0D0E032C0E0C0F0C093
:1000760083C082C0D075D0001242ADD0D0D082D01D
:0600860083D0F0D0E0324F
:00000001FF
